:020000040800F2
:10000000C81D00200101000805550008A13D000899
:1000100039530008C10F00082581000800000000C6
:10002000000000000000000000000000B1650008B2
:100030007B2D000800000000AD5A0008D9680008B8
:100040001B010008695800081B0100081B0100087B
:100050001B0100081B0100081B0100081B01000810
:100060001B0100081B0100081B0100081B01000800
:100070001B0100081B010008A12800081B01000843
:100080001B0100081B01000859070008FD7B000840
:10009000A97C00081B010008E90F00081B010008EB
:1000A00069690008656A00081B0100081B01000857
:1000B000696A0008516D0008AD6F00081B01000857
:1000C0001B0100081B0100081B0100081B010008A0
:1000D0001B0100084D7B00081B0100081B010008E4
:1000E0001B0100081B0100081B010008DFF80CD0F1
:1000F00000F0F4FA0048004739970008C81D0020B6
:100100000648804706480047FEE7FEE7FEE7FEE7B1
:10011000FEE7FEE7FEE7FEE7FEE7FEE7F56800081C
:10012000ED0000082DE9F0410024061B254671F181
:10013000000605DA01240027D0EB070067EB010178
:10014000161E73F1000605DA0027D2EB070201251F
:1001500067EB030300F0DEF986460E4617469C4621
:10016000AC4204D00025D0EB050E65EB010624B1AE
:100170000020D2EB000760EB030C704631463A4694
:100180006346BDE8F08140EA01039B0703D009E024
:1001900008C9121F08C0042AFAD203E011F8013B73
:1001A00000F8013B521EF9D2704710B5002200E062
:1001B000521C835C8C5CA34201D1002BF8D1D8B2D5
:1001C000E1B2401A10BD80EA010210B502F000430E
:1001D000400022D04A001FD0010E01EB1261C0F393
:1001E0005600C2F3560240F4000042F40002A0FBA5
:1001F000022000047F39140400D0401C50EA124051
:1002000001D44000491EC2B20C0604EBD010401CC1
:100210004008802A02D003E0002010BD20F0010039
:10022000002900DA0020184310BD2DE9FE4F81EAB5
:10023000030404F0004421F0004100944FF0000B4F
:1002400023F0004350EA01045ED052EA03045BD07D
:10025000C3F30A54C1F30A552C44A4F2F3340194B5
:10026000A0FB0254C1F3130141F48011C3F3130343
:1002700043F4801301FB024400FB034E840A970AF7
:1002800044EA815447EA8357A4FB076802958D0A24
:1002900005FB07854FEA932C04FB0C542705029DB0
:1002A0004FEA065847EA1637B5EB08056EEB070C20
:1002B000870E920E47EA811742EA8312A7FB0201DA
:1002C000B6EB0B0164EB00042B0D43EA0C335E1814
:1002D00044EB1C50DA465146E7FB0201C5F3130418
:1002E0004FEA0B3343EA14534FEA0432019C43EACA
:1002F0000603A4F10C040294009CCDE900B400F0C4
:100300009FF903B0BDE8F08F00200146F9E72DE921
:10031000F04D81EA030404F0004B21F0004514463F
:100320004FF0000A23F0004150EA050220D054EAC1
:1003300001021DD0C5F30A570246C5F31303C1F3EA
:100340001300C1F30A5640F4801543F48013A7EB61
:100350000608101BD64608F2FD3873EB050002D3E1
:1003600008F1010801E092185B41B8F1000F03DACF
:1003700000200146BDE8F08D00204FF480110646B4
:1003800084460EE0171B73EB050705D3121B63EBC6
:10039000050306434CEA010C49084FEA3000921865
:1003A0005B4150EA0107EDD152EA030012D082EA24
:1003B000040083EA0501084305D0101BAB4106D2B7
:1003C0000122002306E000224FF0004302E06FF01C
:1003D000010253101AEB06004CEB085110EB0A0017
:1003E00041EB0B01BDE8F04D00F01BB970B521F0F9
:1003F000004303430CD0C1F30A550024D5EB040598
:1004000064EB0403D617AD1AB34102DB00200146AA
:1004100070BD201841EB025170BDC10F80EAE07041
:100420000844CA079623002100F0CDB89623002285
:10043000114600F0C8B80EB5C10F80EAE07008445C
:10044000CA07002140F233438DE80E000A460B46EE
:1004500000F0F6F803B000BD0EB540F23341029152
:100460000021CDE900110A460B4600F0E9F803B07F
:1004700000BD00F0004220F00040C10DC0F31600A6
:1004800040F400007F2901DA00207047962903DC40
:10049000C1F19601C84001E096398840002AF4D0A5
:1004A0004042704770B5C1F30A5201F00045002484
:1004B000C1F3130140F2FF3341F480119A4201DA93
:1004C000002070BD40F233439A42A2F2334203DC73
:1004D000524200F05FF800E090402C43F1D04042DF
:1004E00070BDC1F30A5210B5C1F3130140F2FF33DE
:1004F00041F480119A4201DA002010BD40F23343EA
:100500009A42A2F2334203DC524200F043F810BD9B
:10051000904010BD2DE9F05F0546002092469B46B5
:1005200088460646814640241BE028464146474609
:10053000224600F02FF853465A46C01A914110D374
:1005400011461846224600F016F82D1A67EB0108EE
:100550004F4622460120002100F00DF817EB00095C
:100560004E41201EA4F10104DFDC484631462A46F4
:100570004346BDE8F09F202A04DB203A00FA02F14E
:10058000002070479140C2F1200320FA03F3194381
:1005900090407047202A04DB203A21FA02F0002123
:1005A000704721FA02F3D040C2F120029140084383
:1005B000194670470029A8BF7047401C490008BF72
:1005C00020F00100704710B4B0FA80FC00FA0CF083
:1005D00050EA010404BF10BC704749B1CCF12004BB
:1005E00021FA04F411FA0CF118BF01212143084348
:1005F000A3EB0C01CB1D4FEA00614FEA102042BF74
:10060000002010BC704700EBC35010440029A4BF69
:1006100010BC7047401C490008BF20F0010010BC0E
:10062000704710B5141E73F1000408DA401C41F144
:10063000000192185B411A4301D120F0010010BD66
:100640002DE9F04D92469B4611B1B1FA81F202E0DC
:10065000B0FA80F220329046FFF78DFF04460F4635
:1006600040EA0A0041EA0B0153465A46084313D0B8
:10067000114653EA010019D0C8F140025046FFF775
:1006800089FF05460E46504659464246FFF773FF1E
:10069000084305D0012004E020463946BDE8F08D2E
:1006A0000020054346EAE0762C4337430A98630569
:1006B000E40AA0EB08000022FD0A44EA47540A308D
:1006C00002D500200146E9E7010510196941DDE97D
:1006D000084500196941BDE8F04DA2E7064C074DF9
:1006E00006E0E06840F0010394E807009847103402
:1006F000AC42F6D3FFF7FEFC1CB900083CB9000879
:1007000070B58C1810F8015B15F0070301D110F8D3
:10071000013B2A1106D110F8012B03E010F8016B00
:1007200001F8016B5B1EF9D12B0705D40023521E83
:100730000DD401F8013BFAE710F8013BCB1A921CEB
:1007400003E013F8015B01F8015B521EF9D5A142E9
:10075000D8D3002070BD000070B54A4C4FF49065AE
:100760002946204600F017FA002860D02946204686
:1007700000F09EF844490888401C0880012120466A
:1007800000F0E8FA414942F21072B1F85800904284
:1007900002D2401CA1F8580009F004FA3C4DB5F90A
:1007A0001410B5F9120007F0ABFE3A4CA5F856004C
:1007B0002080A16820468847A088A5F8580004F04A
:1007C0000BFF09F0EFFA344E344C307808282FD064
:1007D00045F6AC30606042F6EF60A06042F2C400C3
:1007E000E0602F48008A2080208E6080A16B2B481B
:1007F0008847208E40F21C7180002A4C00EB81005B
:100800006887A2684FF0000550071AD5264840F2C5
:100810001A63C188491C89B2C180994207D3234B0E
:1008200049F68141198022F00401A160C58070BDA4
:1008300041F2130060604FF48060A06040F61B50EE
:10084000CEE730780A2818D2DFE800F01706130543
:100850000A050D171113EAE7BDE8704008F026B845
:100860000AF042FA05E0BDE8704004F039B808F03B
:1008700039FDBDE8704009F0EDBB01F0DFFD84F803
:10088000BA5070BD00240140480700203801002004
:100890004C000020300700203F070020CC00002043
:1008A000F0010020A4020020C80A0020442C0140CE
:1008B0006FEA1121016070470029816802D041F080
:1008C000010101E021F00101816070470029816888
:1008D00002D041F4807101E021F4807181607047A1
:1008E0002DE9F041854E92B0304600F011F90BA889
:1008F00000F03FFA01214FF4C06005F06BF90024CD
:100900008DF831404FF46020CDE90D044FF4A02064
:100910004FF00A080B9001278DF83C808DF830705D
:100920000BA9304600F086F9754D8DF831408DF8F1
:1009300030708DF83C700BA9284600F07BF901233C
:100940001A460F21304600F0C6F902220123114653
:10095000304600F0C0F9012303221946304600F06A
:10096000BAF9012304220021304600F0B4F9012332
:1009700005220321304600F0AEF9012306220821AA
:10098000304600F0A8F9012307220A21304600F082
:10099000A2F9012308220B21304600F09CF9012323
:1009A00009220D21304600F096F901230A22042184
:1009B000304600F090F90121304600F084F9012121
:1009C000284600F080F901231A460521304600F040
:1009D00055F901231A460621284600F04FF9002157
:1009E000304600F0CBF84FF4E041284600F0C6F85E
:1009F0000121304600F0B8F80121284600F0B4F893
:100A00000121304600F0A6F80121284600F0A2F8A6
:100A10000121304600F09EF90121284600F09AF9A4
:100A200040F61451374806F098FD12208DF840002A
:100A300002208DF841008DF842408DF8437010A8D7
:100A400004F08EFD01224FF49061304600F0E8F88A
:100A500001213046FFF73AFF01213046FFF72CFF16
:100A600001212846FFF728FF304600F06EF9304696
:100A700000F09FF80028FAD1304600F075F93046B2
:100A800000F082F80028FAD1284600F05EF92846E6
:100A900000F08FF80028FAD1284600F065F92846C2
:100AA00000F072F80028FAD10121084605F06EF82E
:100AB000154D284601F030FF684601F0D0FF0F4881
:100AC00001A94C300090114881E811018020CDE946
:100AD00004404000069080000790202008904FF4CA
:100AE0004050CDE909046946284601F09BFF0121E9
:100AF000284601F005FF12B0BDE8F0810024014056
:100B000000280140002C014008000240B4020020EF
:100B10000D4910B5884202D1012144150AE00B4964
:100B2000884202D10121041504E0094988420AD112
:100B30000121CC03204605F059F82046BDE81040BD
:100B4000002105F053B810BD0024014000280140E9
:100B5000003C01400029816802D041F4801101E08D
:100B600021F48011816070470029816802D041F42E
:100B7000004101E021F4004181607047826822F465
:100B8000E0420A43826070470146002089684907B5
:100B900000D50120704710B50246002054680B0AAA
:100BA000C9B20C401168194202D0002C00D00120BB
:100BB00010BD014600208968090700D50120704753
:100BC00038B501211C2005F005F8EF20ADF8000034
:100BD00000248DF8034003258DF8025069460D4826
:100BE00002F0E8FC0120ADF800008DF803408DF81C
:100BF00002506946084802F0DDFC3B20ADF80000D9
:100C00008DF803408DF802506946044802F0D2FC8A
:100C100038BD000000080140000C014000100140F8
:100C2000002A4268C9B201D00A4300E08A43426008
:100C30007047000010B542680E4B0C791A400B68E3
:100C400042EA04221343436083680B4A1340D1E90C
:100C5000024222434C7943EA44031A438260C26A47
:100C6000097C22F47002491EC9B242EA0151C162F4
:100C700010BD0000FFFEF0FFFDF7F1FF70B5072487
:100C800009290AD9C568A1F10A0606EB4606B4404F
:100C9000A543B3401D43C56007E0056901EB41066C
:100CA000B440A543B3401D430561836BC3F30154B6
:100CB000121B921C02EB82041F22A2409343A1400C
:100CC0000B43836370BD826B491E22F4401242EADB
:100CD00001518163704770B5072409290AD9C56895
:100CE000A1F10A0606EB4606B440A543B3401D43F6
:100CF000C56007E0056901EB4106B440A543B34078
:100D00001D4305611F23072A09D2446B521E02EBC3
:100D1000820293409C4391400C43446370BD0D2A72
:100D200009D2046BD21F02EB820293409C43914094
:100D30000C43046370BDC46A0D3A02EB8202934017
:100D40009C4391400C43C46270BD816841F008012E
:100D5000816070470029816802D041F4A00101E060
:100D600021F4A00181607047816841F00401816035
:100D7000704700210160017141718160C1600121F2
:100D800001747047002800DA4042B0F5803F02DB72
:100D90004FF6FF70704780B27047000070B51E4C70
:100DA000214694F83800B1F8425006281ED9B4F80C
:100DB0004A10B4F84C00A1EB000202F10902122A19
:100DC00004D8FFF749FB0022144B0AE0884204D202
:100DD000FFF742FB0022124B03E0FFF73DFB00222E
:100DE000104BFFF722FAFFF77CFB09E005D12846FC
:100DF000FFF732FB0C4A0D4BF3E70D4951F8200089
:100E0000C5EB45116063B0EB410F03D9C5EB45104D
:100E10004000606370BD00005804002000003440B2
:100E200000003340000035406766666666E64B406A
:100E3000A0AF000810B50C4C2078400713D5FFF781
:100E4000ADFF0A49A08E088008483038018821F09B
:100E500010010180001F018841F0100101802078FD
:100E600020F00400207010BD580400204004004011
:100E7000F0B4254B002103F134009A793AB1234AAA
:100E800041F2CD05B2F90240AC4211DC99711E4C21
:100E900082683434C2F3C006C2F300252468AE422F
:100EA00011D1240706D5D40506D442F0080205E086
:100EB0009180C162F0BC704722F008028260998282
:100EC000012098711AE090F84A60D6B9104E766CFD
:100ED000B6F5966F15DC240713D49C8AB4F5FA6F27
:100EE00002D2641C9C82E5E70A4B65F3C3021C78BE
:100EF00024F001041C70598019828260F0BC07F054
:100F0000F5BF9982D6E7000070020020E2050020BC
:100F100038010020B00A0020012180F82E104FF483
:100F2000AF6101861F21418645F27151818670476C
:100F300070B506464089204B204C4FF400510025E7
:100F400080B362887AB1012A0CD1E188491C89B248
:100F5000E1803289914205D36580E580FF2801D088
:100F6000401E708170BD70882288904201D9012294
:100F700000E00022184602F0A6FB7088B188014408
:100F80002088401C80B220808142EBD82580A08838
:100F9000401C80B2A080F1888842E3D301206080A9
:100FA000A58070BDFFE70022184602F08CFBA580EB
:100FB000E58025806580F4E700100140C805002029
:100FC000FEE7000010B5074C0021204600F06AF84B
:100FD0000121204600F066F82046BDE810400221BD
:100FE00000F060B80064004010B50D4C0B4920467D
:100FF00000F06AF809492046891C00F065F80949A3
:10100000204600F061F8084C206807F06FFC0021D2
:1010100006A008F0C5FC206010BD00000200F01022
:10102000006400407000F0304C0800206465765F7A
:1010300063616E310000000070B51848017861F3FB
:101040000704417861F30F24817861F31744C17874
:1010500061F31F640179407961F3070560F30F259F
:1010600002F0B0F80E4E304602F054F8A1B230460D
:1010700002F08CF8210CB01C02F088F8A9B2301DE7
:1010800002F084F805482838C07800F00301B01D4C
:1010900002F07CF8BDE8704002F070B8A7070020AD
:1010A00000E4010841B101290AD0022903D1816875
:1010B00041F4000181607047816841F08001F9E7E7
:1010C000816841F40041F5E70A4A914202D10021CA
:1010D00081617047C1F313028B0101D5C260704773
:1010E0004B0101D502617047090101D5826070474B
:1010F000426070477000F03030B50823102404229D
:10110000B1F5007F1DD010DC202929D007DC012992
:1011100021D0042922D0082900D1C46030BD402943
:1011200020D0B1F5807FF9D10BE00025B1F5004F5B
:1011300006D008DCB1F5806F03D0B1F5006FEDD1BA
:101140008561426030BDB1F5803F0DD0B1F5003F03
:10115000F8D1446030BD0549816030BDC36030BD09
:10116000036130BD046130BD436030BD0101010049
:101170003EB5684600F026FA00208DF808000121EF
:101180008DF809108DF80A008DF80B108DF8060007
:101190001D498DF807008DF8020001F11000897CCF
:1011A0008DF80310C1788DF8041001798DF80510C1
:1011B000C088164CADF800006946204600F045F99D
:1011C00001220221204600F038F901221146204672
:1011D00000F033F90E492046FFF776FF0C49204610
:1011E000891CFFF771FF0B492046FFF76DFF084987
:1011F0002046491EFFF768FF01224FF404412046B4
:1012000000F01BF900203EBD5C0800200064004097
:101210000200F0107000F030094910B588424FF01C
:10122000010101D14C0601E04FF08064204604F03A
:10123000C5FC2046BDE81040002104F0BFBC000002
:10124000006400402DE9FF470026012119488DF870
:101250000B608DF80C10DFF86090ADF808608DF829
:101260000D10354634464FF0040809F1800AC7686E
:101270001AE000BF8DF80A4059F82610761C480B7A
:10128000ADF8000008EBC101ADF802105AF82510C6
:101290006D1C4A0BADF8042008EBC100ADF8060048
:1012A000684600F00BF8641CBC42E3DB04B000208D
:1012B000BDE8F08748080020B0180020F0B5827A19
:1012C000012191402E4A136843F0010313602C4B17
:1012D0001C331C688C431C60294D067B294C0C3543
:1012E000A6B92E688E432E604688C78846EA074610
:1012F000877A04EBC707C7F840660688878846EAFE
:101300000746877A04EBC707C7F84466067B012EB9
:1013100012D12E680E432E60867A056804EBC6064D
:101320004FEA3545C6F84056867A456804EBC60450
:101330004FEA3545C4F84456114CC57A241D002D9A
:10134000256806D00D4325600D4C0589143415B170
:1013500004E08D43F7E725688D4325600589012D5D
:1013600002D125680D432560407B012802D1186811
:1013700008431860106820F001001060F0BD000004
:1013800000660040006000400246002053690B42A6
:101390004AD0B1F5807F3BD013DC08292ED007DC82
:1013A000012926D0022927D004293DD1D0682BE07D
:1013B000102925D0202926D0402935D110691021A7
:1013C00030E0B1F5004F2BD00BDCB1F5007F22D01F
:1013D000B1F5806F22D0B1F5006F25D190697021F1
:1013E00020E0B1F5803F11D0B1F5003F1CD150682D
:1013F000E5E790680D4915E0D06802E0D068DEE7C7
:10140000106903210EE0106908210BE05068FBE72A
:101410009069012106E09069022103E0906900E0F3
:101420005068042100F0E4BF704700000101010092
:101430008069C0F3021000017047002A426901D0A0
:101440000A4300E08A434261704710B503680022F6
:1014500023F002030360036843F0010303604FF6C7
:10146000FF7300E0521C4468E40701D19A42F9D1AD
:101470004268D2073ED08A79012A02683CD022F025
:1014800080020260CA79012A026838D022F0400244
:1014900002600A7A012A026834D022F02002026037
:1014A0004A7A012A026830D022F0100202608A7A59
:1014B000012A02682CD022F008020260CA7A012AAE
:1014C000026828D022F0040202608A78CC78920761
:1014D00042EA04620C7942EA04424C79098842EA01
:1014E0000452491E0A43C261016821F001010160F2
:1014F000002114E0002010BD42F08002C1E742F05C
:101500004002C5E742F02002C9E742F01002CDE7F1
:1015100042F00802D1E742F00402D5E7491C4268D4
:10152000D20701D09942F9D14068C007E2D1012029
:1015300010BD000010B500EB0113D3F8B04114F05A
:1015400004041472D3F8B04134D0E408C2F8044063
:10155000D3F8B04104F002045472D3F8B44104F05B
:101560000F049472D3F8B441240AD474D3F8B84168
:10157000D472D3F8B841240A1473D3F8B841240CB8
:101580005473D3F8B841240E9473D3F8BC41D47388
:10159000D3F8BC41240A1474D3F8BC41240C54740D
:1015A000D3F8BC311B0E937439B1016941F02001AD
:1015B000016110BD640D1460CAE7C16841F02001EB
:1015C000C16010BD00218171C171017241728172CF
:1015D000C1728170C1700321017102214171012129
:1015E0000180704730B50246002093685B0108D443
:1015F0009068000101D5012003E09068C00037D554
:10160000022002EB0012D2F8803103F00103C2F88D
:1016100080310B7A73B3D2F880414D681C434B7A0A
:1016200043EAC5031C43C2F880418B7A03F00F03E1
:101630008B72D2F8843123F00F03C2F88431D2F8D0
:1016400084318C7A2343C2F88431CB7ACC6843EA64
:101650000423C2F88831CB7B096943EA0121C2F82F
:101660008C11D2F8801141F00101C2F8801130BD17
:10167000042030BDD2F880314C7A23430C8843EAF1
:101680004453C2F88031D0E72DE9F04FFE481A21CB
:1016900085B0406CB0FBF1F086B20D20B6FBF0FADD
:1016A000FA48FB49B0F91A00C0F30F100490B1F9E1
:1016B0001020C82042434FF47A7000EBA2339CB252
:1016C000092303EBA232132A00D2044689460D46B1
:1016D000B1F91E0001F096F80390B5F9200001F071
:1016E00091F80290B5F9220001F08CF8E94B0190D5
:1016F000D88B4FF4FA71484340F6FF71B0FBF1F01C
:10170000DFF894C31FFA80F8E44DBCF81000E449F8
:101710000090E8880A78070967F30002C70A67F3B0
:101720004102C70867F38202870867F3C302070B09
:1017300067F30412470867F3451260F38612470BFC
:1017400067F3C7120A704A78470A67F3000247092D
:1017500067F34102870967F38202070A67F3C3024E
:10176000C70967F304122F7ABF0867F34512800B8D
:1017700060F386124A7093F8070110B142F08000BE
:1017800001E022F080004870C4489B46827A887845
:1017900062F341001A461B89DD0885EA1325ED43F3
:1017A00065F382009CF8005065F304105D0965F351
:1017B0004510DB0A63F386101388DB135B1C63F3AD
:1017C000C71088709BF84A202AB1012A07D0022A44
:1017D0000AD0032A0DD0CA7822F003020CE0CA789E
:1017E00022F00302521C07E0CA7822F00302921C86
:1017F00002E0CA7842F00302A94BCA702833A3F171
:1018000018059A7802F00302012AAA7812D022F071
:101810001002AA70CA7897070FD020F008008870CD
:101820009F482830407900F00300012808D00228A2
:1018300009D00BE042F01002EBE740F00800EEE7C1
:1018400042F0040001E022F00400C870944F3246D8
:10185000791DF87820F09000F870381D05F038F800
:10186000904EB6F9020005F0E6FEB871B6F9040034
:1018700005F0E1FEF87107F10806711C3046049A84
:1018800005F026F82246F11CB01C05F021F8864828
:101890006421B0F904004843800B03F071F97071C2
:1018A0004246F11DB01D05F013F8B9F91000FFF71D
:1018B00069FAC8214843000C03F062F9287006F168
:1018C0002000012401780227B4EB911F03D1A978ED
:1018D00041F0010105E0B7EB911F03D1A97821F098
:1018E0000101A970437803F00301012902D0022904
:1018F00004D007E0A97841F0020102E0A97821F0C4
:101900000201A970DBF80820A9784FEAD21C6CF319
:101910008201A97090F802C05E46CCF3810CBCF144
:10192000010F03D0BCF1020F03D005E041F020010C
:1019300001E021F02001A9708346A046B4EB931F7B
:1019400003D1C8B240F0800004E0B7EB931F02D18E
:1019500001F07F00A8705548DFF84091504C417F5E
:10196000E878183461F34100D10A61F3820096F8F7
:101970002A1161F30000317961F3C300E87099F82E
:101980000A302979484663F3820133785B115B1C86
:1019900063F3C301530963F30411297111166A79C2
:1019A000491C61F3C3026A7199F80020E97962F376
:1019B0000301C28899F80800D20B62F38611C008AF
:1019C00060F3C711E9715246611C204604F080FFA4
:1019D000E11CA01C009A04F07BFFB6F9E800FFF7B9
:1019E000D1F9C8214843800B03F0CAF82071307A3E
:1019F000C109A07961F3C710B6F8C8100A0A62F3EA
:101A00000600A071E171273C611C2046039A04F096
:101A10005FFFE11CA01C029A04F05AFF611D201D0B
:101A2000019A04F055FF84F806A09BF800005C467C
:101A300020F00C00001D20F03000103020F0C0031A
:101A400040338BF800309BF80100DFF854A020F001
:101A50000300401C20F00C00001D20F0C0024032AA
:101A60008BF80120A078AAF11F0A20F00300401C87
:101A700020F00C00001DA0708346E07820F0E0010B
:101A80004031E17014E0000038010020D004002053
:101A900038050020A4020020B00A0020000C00201D
:101AA0007F070020F80D0020E2050020200E002016
:101AB0009AF8000000287DD0F07B00287AD18AF8BF
:101AC00000000AF1170090F800C00CF0030CBCF104
:101AD000010F06D090F800C00CF0030CBCF1020F0F
:101AE00004D190F800C06CF3010323700378C3F3B2
:101AF0008103012B04D00378C3F38103022B06D1A9
:101B000003784FEA930C23786CF3830323700378F4
:101B1000C3F30113012B04D00378C3F30113022B89
:101B200006D103784FEA131C23786CF30513237056
:101B30000378B8EB931F03D00378B7EB931F06D15C
:101B400003784FEA131C23786CF3871323704378D0
:101B500003F00303012B04D0437803F00303022BAB
:101B600003D1437863F3010262704278C2F38102C9
:101B7000012A04D04278C2F38102022A05D14278B8
:101B80009308627863F3830262704278C2F30112B1
:101B9000012A04D04278C2F30112022A05D1427808
:101BA0001309627863F3051262704278B8EB921FF2
:101BB00005D000E018E14278B7EB921F05D14278DA
:101BC0001309627863F387126270827802F003026D
:101BD000012A04D0827802F00302022A04D1837819
:101BE0005A4663F30102A2708278C2F38102012A8D
:101BF00004D08278C2F38102022A05D18278930848
:101C0000A27863F38302A2708278C2F30112012AE0
:101C100004D08278C2F30112022A05D18278130916
:101C2000A27863F30412A2708278B8EB921F03D0FB
:101C30008278B7EB921F06D18278C2F30113A278A3
:101C400063F34712A270C278D20608D0C27802F0BD
:101C50001F021F2A03D2C27862F30401E170C17827
:101C6000490905D0C1784A09E17862F34711E1706A
:101C7000017901F00301012904D0017901F0030188
:101C8000022904D10179227961F3010222710179DB
:101C9000C1F38101012904D00179C1F38101022935
:101CA00005D101798A08217962F3830121710179D3
:101CB000C1F30111012904D00179C1F301110229F5
:101CC00005D101790A09217962F3051121710179A0
:101CD000B8EB911F03D00179B7EB911F05D10179C2
:101CE0000A09217962F387112171417901F0030119
:101CF000012904D0417901F00301022904D141797D
:101D0000627961F3010262714179C1F381010129B4
:101D100004D04179C1F38101022905D141798A08B2
:101D2000617962F3830161714179C1F30111012984
:101D300004D04179C1F30111022905D141790A0981
:101D4000617962F3051161714179B8EB911F03D09C
:101D50004179B7EB911F05D141790A09617962F3A5
:101D600087116171817901F00301012904D0817922
:101D700001F00301022904D18179A27961F3010202
:101D8000A2718179C1F38101012904D08179C1F364
:101D90008101022905D181798A08A17962F3830141
:101DA000A1718179C1F30111012904D08179C1F3B5
:101DB0000111022905D181790A09A17962F305117E
:101DC000A1718179B8EB911F03D08179B7EB911F95
:101DD00005D181790A09A17962F38711A171C179CD
:101DE000E07961F30300E071434F387800F00F00B1
:101DF000042801D1FFF720F92078C0F381000128E1
:101E000039D1F879010636D500F07F00142832D890
:101E1000A87840F00400A870384AA978107F8B0792
:101E20004FF47F412BD5802821D3354B00F01F0084
:101E3000126853F82000024219D1B06840F0807057
:101E4000B0602D4830388078C0071CD0B068C00121
:101E500019D52C48406C322815D85446BAF80200DF
:101E60008A46504527D101F04BFC60800DE0B068F8
:101E700020F08070E4E7A87820F00400CBE7B06899
:101E800020F08070B060AAF80210A878800702D411
:101E90000020A9F80A003879C00701D0A9F80A8003
:101EA00099F80A00C1071448A0F14900017812D03E
:101EB00041F0010111E001F00BFC40F6B83188421D
:101EC000E3D3B068C101E0D50005DED4A9F80A80EB
:101ED000A4F802A0D9E721F001010170B168C9019D
:101EE000017802D541F0020101E021F00201017008
:101EF00005B0BDE8F08F0000AF070020E805002026
:101F000000B400083801002070B51548006810F0D2
:101F1000E05F23D0134CD4E9001081421ED004EBC3
:101F2000001104F5A1608A6842600A7B8272042372
:101F30000372002545720B300E31FEF724F972B69C
:101F40006068401C6060402800D3656062B6064946
:101F5000BDE8704002480838FFF744BB70BD000080
:101F600008640040A8140020B0190020FCB5054604
:101F70004FF6FF7600200C46ADF8006048F20507EA
:101F80008DF8040020E000BF15F8010B8DF8040067
:101F900001A9084602F080FBBDF800009DF804107E
:101FA00080EA0120ADF800005FF00000BDF80010ED
:101FB0000A0402D587EA410101E006EA4101401C1A
:101FC000ADF800100828F1DB641EDDD26946084632
:101FD00002F04CFBBDF80000FCBD000002460020F2
:101FE00004E000BF12F8013B1844C0B2491EF9D208
:101FF0007047000070B5144A85B01088002413495A
:1020000001940094039420460494138807E0CD8B38
:10201000009E354400950D8B019E35440195158831
:102020009D42F4D0401CC0B28028EED300984111EC
:1020300007484180848001984111064881830183CB
:10204000818205B070BD000048070020A402002076
:10205000E2050020D004002030B4104C00200346DC
:102060004FF47F42A4F1340121F8103024F81020FD
:10207000401C1A28F8DB0A4B002000BF33F8104040
:1020800021F81040401C1A28F8DB06480649028057
:10209000012081F8300030BC03F050B96C100020F2
:1020A000080800203C080020CC0E00202DE9F84351
:1020B00003F090F9C64DC54B00204FF47F4105F168
:1020C000340400BF35F8106033F81020964203D076
:1020D00025F8102024F81010401C1A28F2DBBD4807
:1020E00090F83000012808D05FF0000024F81010AC
:1020F000401C1A28FADBBDE8F88302F0F1FD2088C5
:1021000001F0E6FA2988B44E88420AD301F0F8FAC1
:102110002080B24800906B460822B149306808F030
:10212000A5FE608801F0D4FA698888420CD301F0DA
:10213000E7FA6080A948AA49401C00906B46082233
:102140000831306808F092FEA08801F0C1FAA98831
:1021500088420CD301F0D4FAA080A048A049801C8A
:1021600000906B4608221031306808F07FFEE0884E
:1021700001F0AEFAE98888420CD301F0C1FAE080A0
:1021800096489749C01C00906B4608221831306869
:1021900008F06CFE208901F09BFA298988420CD353
:1021A00001F0AEFA20818D488D49001D00906B46EC
:1021B00008222031306808F059FE608901F088FA61
:1021C000698988420CD301F09BFA60818348844975
:1021D000401D00906B4608222831306808F046FE0A
:1021E000A08901F075FAA846A98905277D4D884286
:1021F00016D36878052813D201F082FAA081687896
:10220000401CC0B26870052800D96F7073487449CB
:10221000303000906B4608223031306808F026FEDE
:10222000E08901F055FAB8F80E10884216D3A87864
:10223000052813D201F064FAE081A878401CC0B2EE
:10224000A870052800D9AF70644865493130009006
:102250006B4608223831306808F008FE208A01F009
:1022600037FAB8F81010884216D3E878052813D248
:1022700001F046FA2082E878401CC0B2E8700528D8
:1022800000D9EF7055485649323000906B4608220D
:102290004031306808F0EAFD608A01F019FAB8F8B8
:1022A0001210884216D32879052813D201F028FA93
:1022B00060822879401CC0B22871052800D92F718E
:1022C00046484749333000906B4608224831306811
:1022D00008F0CCFD208D01F0FBF9B8F82810474636
:1022E00088420BD301F00CFA20853F483C4900900E
:1022F0006B460822A031306808F0B8FD608D01F00F
:10230000E7F9798D88420CD301F0FAF960853648F7
:102310003349401C00906B460822A831306808F011
:10232000A5FDA08D01F0D4F9B98D88420CD301F040
:10233000E7F9A08529482A49503000906B460822C9
:10234000B031306808F092FDE08D01F0C1F9F98DEF
:1023500088420CD301F0D4F9E08520482049603050
:1023600000906B460822B831306808F07FFD208E5F
:1023700001F0AEF9398E88420CD301F0C1F9208604
:1023800016481749613000906B460822C03130680A
:1023900008F06CFD608E01F09BF9798E88420CD3B9
:1023A00001F0AEF960860D480D49623000906B4631
:1023B0000822C831306808F059FD0C48FFF738F89A
:1023C00000283FF498AE287095E600000808002029
:1023D00038100020CC0E00204C0800200002FF180E
:1023E000000F0020400800200006FF180064004095
:1023F000024600200A4200D00120704730B50E4945
:1024000002880A800C4A4388083A13800B1F808890
:1024100018802024151F2C800020401C80B23C28EE
:10242000FBD341F69910088044F64800108046F628
:10243000480018802C8030BD202C0140114944F602
:1024400048000880091D46F648000880091D41F62D
:10245000991008800B48001F018841F0200101807D
:1024600009480021A0F86810A0F86610A0F86410D0
:10247000A0F86210A0F86010A0F85E100348418137
:1024800081827047182C0140A40200204C000020DB
:102490002DE9F04F4B4B4C480021DA7A0678802A20
:1024A00026F001057AD31C68484B02F01F0253F84E
:1024B0002220474B14421A6802D042F0200201E069
:1024C00022F020029946DFF80CB11A60434B404FCE
:1024D0009BF80040DFF800A1B3F9043097F84AC038
:1024E000022C5CD1D9F80870C7F3C004C7F30028E8
:1024F000444554D0364C343C94F80280B8F1000F77
:1025000006D0B8F1010F0DD0B8F1020F4CD120E088
:10251000110549D5910647D40121A17026F0040187
:10252000017041E015053FD495063DD575073BD4B4
:10253000458895BB4380002B09DD46F005010170FD
:102540000221A1702649B1F8441001822CE0A1704B
:102550002AE0C6880EB9002B14DC067B664511D133
:10256000204EB6895FEA46780CD45FEA867809D4B3
:102570005FEA427806D55FEA826803D5F60701D1A3
:10258000FE0111D505704180AAF800104181018239
:10259000A17089F80F108BF8001005E00EE00570AF
:1025A0004180AAF800104181C38080F80CC0500916
:1025B00060F3CB22C9F80020BDE8F08F05704180A0
:1025C0004181F9E7E8050020B00A002000B40008C6
:1025D000A40200203F0700200C010020E20500209B
:1025E00038010020000C00202DE9F04796B00024AF
:1025F0000C940D940E940F9472B67C48816941F44A
:1026000000718161816941F4806181614FF4004012
:1026100003F0B2FA764D00212846FEF757F9002163
:102620002846FEF749F9734E00213046FEF744F97B
:10263000714F0021384600F063F901204FF47041DA
:10264000401C8842FCD32846FEF762FAB146304669
:10265000FEF75EFA3E46384600F05EF94FF4602021
:10266000CDE912048DF8454001204FF004088DF8A3
:10267000440010948DF8508010A92846FEF7DAFA2D
:1026800001231A4605212846FEF725FB01230222D5
:1026900006212846FEF71FFB0123032207212846B7
:1026A000FEF719FB012304220F212846FEF713FB36
:1026B000304600F031F9684600F0D1F94C484F4FF0
:1026C0004C300090CDF80C80CDE901748020CDE92C
:1026D00004404000069080000790202008904FF4AE
:1026E0004050CDE909046946304600F09BF90121CC
:1026F0002846FEF7EBF80121304600F001F90121F0
:102700002846FEF7D9F847F2305015941599491C20
:1027100015918142FAD301212846FEF71BFBADF843
:102720002C40B84640F2DC5A4FF4007723E0504684
:1027300015941599491C15918142FAD3B8F80020D7
:102740000D9911440D91B8F802100E9A11440E9192
:10275000B8F804100F9A11440F91B8F806000C99BC
:1027600008440C9001212846FEF7F4FABDF82C002D
:10277000401CADF82C00BDF82C00B842D7D30D9802
:10278000C1111E480A3001830E99C91141830F9966
:10279000C91181830C99C911818000212846FEF757
:1027A00095F80021304600F0ABF800212846FEF7EE
:1027B00083F800214C464846FEF77EF80220C1020D
:1027C000401C8842FCD32846FEF7A2F92046FEF7BB
:1027D0009FF9304600F0A0F8FEF782F808493C2047
:1027E000087062B616B0BDE8F08700000010024025
:1027F0000024014000280140080002402E0500206E
:102800003C07002010B5FEF7BDFAC8214843800BF5
:1028100010BD000070B5204B40F6C81441F2B7055A
:102820005B6C48F6E6065C4305EBA4341B4D734332
:102830004EF6F61606EBA333C5E90443D460401AFE
:10284000536110609168884202DA4942884200DC94
:10285000116010684343107E0341906A1918916219
:10286000506A814200DD9062916A106A814201DB08
:10287000084600E09062A86111684C43117C0C414D
:1028800008412118B2F91C00884204DBB2F91A0091
:10289000884200DC08B270BD38010020140100201D
:1028A00010B54FF40054204600F0ACF8002813D0C7
:1028B0000A49087840F008000870204600F014F833
:1028C0000021074800F01CF80648C17E012903D109
:1028D0000021C1760121017710BD00008206002091
:1028E00044000240040D0020C10002D502490860E6
:1028F00070470249486070470404024000000240EB
:102900000029016802D041F0010102E04FF6FE7299
:10291000114001607047000001684FF6FE721140DF
:1029200001600021016041608160C1603149314A2C
:102930000839904203D1486840F00F0006E02D4A64
:102940001432904204D1486840F0F000486070476B
:10295000284A2832904203D1486840F47060F5E775
:10296000244A3C32904203D1486840F47040EDE77D
:10297000204A5032904203D1486840F47020E5E785
:102980001C4A6432904203D1486840F47000DDE78D
:10299000184A7832904203D1486840F07060D5E719
:1029A000154A111F904203D1086840F00F0006E05D
:1029B000114A1432904204D1086840F0F0000860D7
:1029C00070470D4A2832904203D1086840F4706085
:1029D000F5E7094A3C32904203D1086840F4704060
:1029E000EDE7054A50329042EAD1086840F4702081
:1029F000E5E700000800024008040240406880B299
:102A00007047000001460020CA0001D5034A00E0DB
:102A1000034A12680A4200D00120704700040240B5
:102A20000000024030B5036847F6F07293430C6A29
:102A30008A682243D1E904452C4322438C6922430E
:102A4000CC6922434C6A22438C6A22431A430260B7
:102A5000CA6842600A6882604968C16030BD00216E
:102A6000016041608160C160016141618161C1615A
:102A7000016241628162704710B5114C8CB0002137
:102A80002046FFF73DFF2046FFF746FF0D48009028
:102A90000D480021CDE901016420CDE9030180202A
:102AA000CDE905010791089109910A9169462046EF
:102AB000FFF7B8FF01212046FFF722FF0CB010BD41
:102AC0005800024004380140F0080020F0B540F6FC
:102AD000AA222A49C284838B0C88E31A9BB20F2B4B
:102AE0000DD309888183037E00213BB1244BB3F9C8
:102AF0000A40244B062C03DA818429E08184F0BD4E
:102B0000214C2478022C02D0002CF5D0F0BD1F4CB3
:102B100040F68B27656C1B4CA5F22D16BE42B4F90E
:102B2000004017D2418B491C89B241836429EDD3FF
:102B300064214183B0F92410914201DA01EB2212A1
:102B40008284641C20B24FF4007118808842DDDB5F
:102B50001980F0BD41F29416B542FADBB0F9245069
:102B6000002D02DDA5EB221200E0002282844183C9
:102B7000641E20B218800028EADDF0BD480700205E
:102B80004C000020540400203F07002038010020A2
:102B900010B50446B0F9020043F699114843811379
:102BA000E06840F26662504301EBA030E060B4F9A7
:102BB000001043F6991251438A13216940F266636B
:102BC000594302EBA131216105F03AFC6061A18813
:102BD00040F6AB2208444010A0F515415539E0629B
:102BE000914205D9A0F5F851FF39521C91421DD2EE
:102BF00049F25451884202DDA0F5204002E0A0F5E0
:102C0000F850FF38206300EB400040F34F00208570
:102C1000B4F924104A42904201DA104602E0884298
:102C200000DD0846E083228461848AE0A0F5FE424C
:102C3000FF3A41F255518A4214D8A2F6AA202063E5
:102C400000EB400040F34F002085B4F924205142AE
:102C5000E183884201DA084602E0904200DD104636
:102C6000404250E0A0F5D442AA3A8A4215D2A2F6D8
:102C7000AA20206300EB400040F34F012185B4F906
:102C800024004242E2832084914201DA104602E0AD
:102C9000814200DC0846608453E0A0F5AA42543A21
:102CA00041F256539A4215D2A2F6AB20206300EBB4
:102CB000400040F34F002085B4F924104A4290426E
:102CC00001DA104602E0884200DD08464042E08317
:102CD000218419E0A0F5804241F254539A4215D262
:102CE000A2F6AA20206300EB400040F34F002085AD
:102CF000B4F92410E1834A42904201DA104602E01E
:102D0000884200DD0846208462841AE0A0F528523B
:102D1000AB3A8A4215D2A2F6AA20206300EB40000B
:102D200040F34F012185B4F92400E083424222841C
:102D3000914201DA104602E0814200DC084640423E
:102D4000A9E7B4F91E0041420948B0F90000414327
:102D50008913E180B4F9201049424143891321814C
:102D6000B4F92210494241438813608110BD00002C
:102D70005404002001210176704770471548164A17
:102D80004FF480410078042821D002F13C03D08A1E
:102D90009B88C01A00B22F2801DD001108E000282E
:102DA00001DD002007E00D4B984201DA184602E0F1
:102DB000402800DD40209389184400B2884203DC9B
:102DC00040F26661884200DA08469081704791813E
:102DD000704700003F070020D0040020C0FEFFFF26
:102DE00038B54B484B4902880B889A1A92B20F2A81
:102DF00071D30988484C01804FF0FF01E2884FF4FD
:102E00007A7355044FF4967002D51622009103E0B0
:102E1000950403D515220091014670E0D50402D532
:102E200014220091F8E7150502D513220091F3E76B
:102E3000550502D512220091EEE7950502D5112223
:102E40000091E9E7D50502D510220091E4E71506C7
:102E500002D50F220091DFE7550602D50E22009120
:102E6000DAE7950602D50D220091D5E7D50602D501
:102E70000C220091D0E7150702D50B220091CBE779
:102E8000550702D50A220091C6E7950702D5092207
:102E90000091C1E7D20702D008220091BCE7228945
:102EA000550702D507220091B6E7950702D50622FD
:102EB0000091B1E7D20702D005220091ACE7A27AD7
:102EC000D20702D004220091A6E7A289D40603D536
:102ED00003220091A0E719E0140702D50222009115
:102EE0009AE7540703D4940701D4D20702D00122F1
:102EF000009191E70020034602460146009003F04E
:102F000003FCBDE838400248FEF712B838BD0000A7
:102F1000F40B002048070020000C0020F0B55948B1
:102F2000594982880B889A1A92B29C2A64D30988DC
:102F3000818056490A880146002A0B7843F0020135
:102F400056D11646524A1C0715680246127822F0DE
:102F5000020274D54F4C0746E4887F785FEA845CB0
:102F600002D547F0010701E027F001074770A704E9
:102F7000477802D547F0020701E027F002074770C3
:102F8000670401D4E70703D0477847F00807477084
:102F9000640603D5447844F0040404E01C0603D41A
:102FA000447824F004044470EC0450D4354C9A075F
:102FB000247824F0100423D4324D42782F7A2D78CF
:102FC000012A45F0100514D0022A16D02D4C042AEF
:102FD000A47804F1010C0CF0FF0C13D0072A25D0C3
:102FE000032A23D0052A21D0062A1FD021F0100160
:102FF00042E0B90702E00570F0BD39070029FADBAD
:103000000470F0BDFA0601D41A060AD50170022C2C
:1030100004D280F802C0BCF1020FF2D341F080016B
:103020002AE021F0100101708670F0BD877A7F06DA
:10303000F7D5032C04D8017080F802C0F0BD0FE072
:103040005107D8D51906D6D443F0800114E0027098
:103050004178CB0701D18907F0D522F010010BE0B0
:10306000E9040BD49907E9D4818AC82902D2491C02
:103070008182E3E743F00A010170DFE70270868294
:10308000DCE7000010070020480700204A07002066
:10309000A4020020000C002070B51148114C4FF024
:1030A0000005C088810503D4410601D4C00515D5AB
:1030B0004FF480610C4800F0FBFA68B9A08840F634
:1030C000B831884201D2401CA08080B2B0F57A7F2E
:1030D00001D30120607070BDA58070BD6570FBE7F5
:1030E000000C002060070020000C0140084946F653
:1030F00068000880091D0880091D41F6DD50088020
:103100000348001F018841F0200101807047000042
:10311000182C014070B50D4E0546304600F05EF8A3
:10312000042811D10A4C206940F002002061656139
:10313000206940F040002061304600F04FF82169DE
:1031400041F6FD721140216170BD0000FFFF0F00CC
:103150000020024008490420CA68D20701D001209B
:103160007047CA68520701D502207047C968C9066E
:10317000FBD503207047000000200240024801698F
:1031800041F080010161704700200240F0B5064621
:103190004FF6FF770D46384600F020F804280DD191
:1031A000074C206940F0010020613580384600F06E
:1031B00015F8216941F6FE7211402161F0BD000051
:1031C00000200240034802494160034941607047C2
:1031D0002301674500200240AB89EFCD00B50346CF
:1031E000FFF7B8FF03E000BFFFF7B4FF5B1E012845
:1031F00003D0002B00D1052000BD002BF4D1FAE74D
:1032000010B5C28800210AB1032206E002890AB182
:10321000022202E0428912B10122027000E0017034
:1032200004784FF4804344F6206244B1012C06D068
:10323000022C07D0032C01D14180818010BD438036
:10324000828010BD41F23331418040F6B731F4E75E
:10325000401A10609168884202DA4942884200DCD4
:10326000116051691068137E41431941936A0B4400
:103270009362516A8B4200DD9162936A116A8B42BC
:1032800000DA9162D168936A4143107C01410341A5
:10329000B2F91C001944884204DBB2F91A008842D2
:1032A00000DC08B270470000054920B1086940F011
:1032B00080000861704703484860034848607047D1
:1032C0000020024023016745AB89EFCD06494FF44A
:1032D0007A70CA68D20705D0401E0004000CF8D1ED
:1032E000FF20704700207047002002400E4A032054
:1032F000A2F14C0182F83E000020C8800B490886EC
:10330000C862C8830884488490620948016DB1F599
:10331000206F01DBA3219162807A002802D0906A9D
:1033200040429062704700004C00002038050020A9
:1033300038010020F0B53D4988894A89801A80B259
:103340000F286AD388894881CA8939480B3A272AC5
:1033500026D28A7822BB8268384B42F4807282601F
:10336000344A374C374D12785607334A0AD4364E12
:1033700036881680354A12881A80354A128822808B
:10338000344A09E0344E36881680344A12881A804E
:10339000334A12882280334A12882A8001228A7096
:1033A000314A0021314B82F84D1019469A7F304D39
:1033B0000968802A32D302F01F0255F822201142F8
:1033C0002CD0826822F48012184E82601236144685
:1033D0001215B778521C62F38617264AB77093F815
:1033E00016C01778BCF1800F27F0020608D30CF046
:1033F0001F0C55F82CC011EA0C0F01D147F0020642
:1034000016701A7E802A0DD302F01F0255F8222072
:10341000114207D144F400218160F0BD826842F47A
:103420008012D1E724F40021F6E700003C070020D9
:10343000A402002038010020C8040020CA04002093
:10344000CC040020CE040020B8040020BA040020E0
:10345000BC040020BE040020C0040020C2040020E0
:10346000C4040020C6040020580E0020E8050020F7
:1034700000B40008D004002070B521488189028979
:10348000891A89B20F2932D381891E4D1E4C0181C0
:10349000697A22681D4E42F00400802908D301F0A9
:1034A0001F012B6856F821100B4201D122F00400B5
:1034B0002060FFF7F1FDA87B802819D300F01F00E2
:1034C000296856F82000014212D1206820F002003D
:1034D0002060E87A80280FD300F01F00296856F892
:1034E0002000014208D1206820F00800206070BD53
:1034F000206840F00200EBE7206840F00800F5E7A4
:103500003C070020E8050020A402002000B40008C9
:1035100030B5044600204FF40043024640EA030160
:1035200001FB01F5A54200D80846521C5B0812B207
:10353000102AF3DB30BD0000F0B51D4C1B4A4FF0E4
:10354000010C94F83B5094F80AE0144692F83C3091
:1035500094F838402B43651CEEB2154D95F83D703C
:103560000025BEF1FF0F0AD0BEF1000F06D18B423D
:1035700013D155700C2C01D282F83860F0BD834213
:1035800002D182F801C0F5E78B42F7D15570B80738
:1035900009E000BF82F83850F0BD8342FCD1F84307
:1035A00082F801C080070028F4D0F0BD5804002044
:1035B00038010020F0B5CA78002502F00F03D206CA
:1035C00001D58A7813430A784FF00F0E12F0FF0FDF
:1035D0004FF001021CD004680F8802FA05F637404C
:1035E000B74211D14FEA850C0EFA0CF724EA07070F
:1035F00003FA0CF43C43CF78282F02D0482F02D096
:1036000002E0466100E006616D1C082DE4D3046011
:103610000C88FF2C1ED944685FF0000606F10807ED
:1036200002FA07F50F882F40AF420FD14FEA860C00
:103630000EFA0CF7BC4303FA0CF73C43CF78282F63
:1036400000D14561CF78482F00D10561761C082E46
:10365000E4D34460F0BD0000F0B5144C002801DA5A
:10366000E36900E06368420D120185B2C0F30157BF
:103670009540C0F30346032F05D0C2020AD50322AA
:10368000B240934307E023F07062636823F07063F5
:10369000636002E0AB4343F0706201B12A4300284B
:1036A00001DAE261F0BD6260F0BD0000000001409F
:1036B0000246002092680A4200D001207047416112
:1036C0007047016170470AB10161704741617047FD
:1036D0004FF6FF62B0F57F4F04D0911C884203D1B2
:1036E000002070471046704704490988814201D381
:1036F000081A01E0101A084480B2704788080020B8
:103700000148008870470000880800200F4A104BCD
:1037100092F838105B5C834201D1012004E00D4B2C
:103720005B5C834203D1002082F83A0070470A4B69
:103730005B5C834201D18120F6E7084B595C8142F2
:1037400001D18020F0E70320EEE7000038010020DF
:10375000B8B80008CAB80008BEB80008D0B8000859
:103760000A4810B501784FF000024C0708494FF0A5
:10377000FF0389684FEA017105D5002901DA8272D9
:1037800010BD837210BD0029FBDBF8E73801002073
:10379000A4020020F0B5194E194C0022E31CA6F13A
:1037A000060CB75CA518ED78FF5C0D430F43BD42D6
:1037B0001FD01CF80270FF5C0F43BD4219D01546A4
:1037C0000023A618F6780E43C6545B1C1CF8022092
:1037D000DBB2062BF5D3C17881700179C17000216D
:1037E0004218491C15711CF80550C9B20629F7D3B7
:1037F000F0BD521CD2B2032AD3D3F0BD92AF000861
:103800005804002010B502460021064B06205C1823
:103810006478944200D10846491CC9B20629F6D3FF
:1038200010BD0000380100200548D0E900218A427F
:1038300002D14FF0FF30704700EB011080687047F5
:10384000A010002070B5164C05464FF0FF36D4E9A5
:103850000010814221D004EB00108068686060682D
:1038600004EB0010007B00F00F02AA720420287203
:10387000606804EB001105F10B000E31FCF783FCCE
:1038800072B66068401C6060402801D30020606010
:1038900062B6A87A08B1002070BD304670BD000045
:1038A000A010002070B526484FF000028078C107B4
:1038B00024483FD024498988E1BB2449234B4FF455
:1038C000FA65496CB3F87630A94231DD90F84A10B8
:1038D00071B31F49C9790C062AD501F07F015A2915
:1038E00026D290F82B11491CC9B280F82B11C82997
:1038F0001ED380F82B21D0F83041014604F1640634
:1039000091F82C11B34203DD052908D2491C01E0CE
:1039100041B1491E80F82C11C9B2052902D30121F9
:1039200080F82A11191B074C343CE162C0F8303191
:10393000AB4203D280F82A2180F82C2170BD000010
:103940008F070020A4020020E2050020380100209B
:10395000AF0700204FF42032C260002181620E22A6
:10396000028241F262024261082202834FF4604205
:10397000428381834FF07842C0E9082140F6C411A8
:1039800001807047B0F90010B0F90220891A416037
:103990004269037E4A431A41836A13448362426A3E
:1039A000934200DD8262836A026A934200DA826295
:1039B000C268836A4A43017C0A410B41D118B0F9BD
:1039C0001C208A4201DA10467047B0F91A0088427A
:1039D000FADC08B27047000010B514481449B0F87A
:1039E00094200B889A1A92B2B2F5437F1DD90988A8
:1039F000A0F89410B0F8921020F8601F00224286C0
:103A00000C480D4CC2888280C180C389838124897F
:103A1000891AA4B2C4818160E11A0161074A818ACE
:103A2000C182928A8282511A816110BD38010020C0
:103A300048070020200E0020380500204C00002000
:103A400009480A49B0F8B2200B889A1A92B241F696
:103A500084639A4206D3098820F8B21F4188818086
:103A600000214180704700003801002048070020F5
:103A70000D480178C90702D00C49098801E04FF6CA
:103A8000FA71416609490120103908800748243835
:103A9000018841F00101018004481838018821F0B3
:103AA0001801018070470000380100202404004004
:103AB0000A49D1F8982012B1521EC1F8982031F865
:103AC000922F521C21F81A294A6A521C4A628A8F84
:103AD000521C8A8701F8400C704700003801002012
:103AE0001CB52D4890F83B3090F83C20934252D0C2
:103AF00000248DF8044053408DF800309DF80030CC
:103B00000122012B08D09DF80030022B09D09DF82E
:103B10000030042B0AD00DE01F498DF804204431F9
:103B200008E01D498DF80420463103E01A498DF85C
:103B3000042048319DF80420012A2CD190F83D3012
:103B40009DF80040154AA34217D090F83E309DF8EA
:103B50000040234208D0B0F84C30A0F84A300B881F
:103B60001488E31AA0F84C3090F838302BB1B0F834
:103B700040301488E31AA0F8423012880A80A0F876
:103B8000402010F83E1F9DF80020114300F8011955
:103B90009DF8001001701CBD58040020480700204B
:103BA00070B5344D40212846FFF782FD8400802106
:103BB0002846FFF77DFD44EA4004A9152846FFF793
:103BC00077FD0443E1B22C4C94F878508D4250D0EC
:103BD0004D4084F87810012D03D0022D01D0042D22
:103BE00047D194F87C00A84384F87C0094F87B20AB
:103BF000AA420FD084F87B5094F87A2001238B409E
:103C00001A4207D11A4384F87A2094F87910491C93
:103C100084F8791094F87910042928D330B1012858
:103C200011D002280FD004280DD012E01348C1880B
:103C300021F04001C1802078002184F83B1020F061
:103C40006000207005E0217841F02001217084F8A7
:103C50003B000B4994F83B0091F82720904204D098
:103C600081F8270007492020087000F00DF884F83B
:103C7000545070BD0010014038010020000C00209D
:103C8000580E00203C07002070B50D4D40212846FD
:103C9000FFF70EFD840080212846FFF709FD44EA66
:103CA0004004A9152846FFF703FD044305480721F2
:103CB00000F8784F0171002141708170C17070BDB2
:103CC000001001403801002070B5344890F83A10D7
:103CD000CA43920761D001F0030280F8392090F8BE
:103CE0003D305B061B0E80F83D30012A01D0812A51
:103CF00002D15B1C80F83D300278D2074DD0DBB298
:103D000003F00102C3F34004A24246D1B0F856408A
:103D10000025641CA0F85640204CA0F8585090F89C
:103D20003E60A47AB24202D080F83E200DE0A607A1
:103D3000B6EB837F02D080F83F5006E090F83F302A
:103D4000642B02D25B1C80F83F3090F84030642B2B
:103D50000CD25B1CDBB280F84030022B06D204F0A0
:103D60000103934202D1022280F84020012901D0B0
:103D7000002912D190F83820416E00EB8202916147
:103D80000163D0E906121144D0E908231A44114412
:103D9000826A1144C26A1144416370BD3801002037
:103DA000FEE700002DE9F04F00BF00209E4E9F4A25
:103DB000A6F51271A6F5BE79A6F1440B06F1440EE4
:103DC000804601F5E074A1F1780301F5457A1D5CA8
:103DD00015F0C00706D0402F51D0C02F77D0802FCC
:103DE00076D004E115F01F0504D0154440F080079B
:103DF0002F7201E082F80880012826D0022824D002
:103E0000032822D0042820D008281ED010281CD037
:103E1000874D55F820C0DCF8005054F820703D4024
:103E2000CCF80050824D55F820C0DCF8005056F810
:103E300020703D43CCF800501D5CAD0659F8205071
:103E40002F6813D53AF810C03EE051F820502F6883
:103E500054F820C007EA0C072F6051F820502F6853
:103E600056F820C047EA0C072F60E5E7DFF8B8C135
:103E70000CF1F00C5CF820C007EA0C077EE015F0AE
:103E80001F0504D0154440F080072F7201E082F82E
:103E9000088001281DD002281BD0032819D004282F
:103EA00017D0082815D0102813D0614D55F8205090
:103EB0002F6854F820C007EA0C072F605C4D55F8B6
:103EC00020502F685BF820C047EA0C0756E00BE053
:103ED00056E051F820502F6854F820C007EA0C072C
:103EE0002F6051F82050ECE715F01F0505D0154460
:103EF00040F0800785F8217001E082F821800128D8
:103F000025D0022823D0032821D004281FD0082838
:103F10001DD010281BD0464D55F820C0DCF80050AD
:103F200054F820703D40CCF80050414D55F820C069
:103F3000DCF800505EF820703D43CCF800501D5C6A
:103F4000AD0615D53A4D3AF81070CC3514E051F85D
:103F500020502F6854F820C007EA0C072F6051F852
:103F600020502F685EF820C047EA0C072F60E6E774
:103F70002D4D3AF81070E03D55F820502F6036E096
:103F800015F01F0505D0154440F0800785F8217015
:103F900001E082F82180012830D002282ED00328A9
:103FA0002CD004282AD0082828D0102826D0204D2C
:103FB00055F820C0DCF8005054F820703D40CCF893
:103FC00000501B4D55F820C0DCF80050164F8837C4
:103FD00057F820703D43CCF800501D5CAD06B1D4BD
:103FE000114F3AF81050E03F57F820703D60401CE8
:103FF000C0B21128FFF4EBAEBDE8F08F51F82050AD
:104000002F6854F820C007EA0C072F6051F82050A1
:104010002F68DFF814C00CF1880C5CF820C047EA68
:104020000C072F60D9E700008CB60008E8050020D7
:1040300088B400084FF40771C1824FF458610183BE
:1040400040F6145181837047F0B5C48AB0F900601E
:104050008681B0F90250C581B0F9043002270021F1
:1040600001220382AB4204DBB54202DDC7804281FC
:104070000CE0B34204DBAE4202DDC78041811CE0AC
:104080009D4205DBB34203DDC2804781018115E01B
:10409000B54204DB9E4202DDC280418105E0AE42B2
:1040A00005DB9D4203DDC1804281078106E09E421F
:1040B00004DBAB4202DDC18047810281C3884589B0
:1040C00000EB430700EB4505BB89AE899B1B0FFA4C
:1040D00083FEA0F812E00689AB8900EB460CBCF821
:1040E0000CC0A3EB0C038382B0F91830B7F90CC0F5
:1040F000A3EB0C0CB4EB4C0F04DA80F82010A3F106
:10410000A10113E0A64503DD80F82010B9890BE07A
:1041100026B1012E04D0022E10D004E0062100E0CA
:10412000052180F82010A989091B6D31418309B24E
:10413000B1F5586F04DB5B1E438304E00421F0E714
:10414000002900DC4283418B8183F0BD0B490022B2
:1041500088760A62CA614A62094A32F9103002EB73
:1041600040028B62B2F90220CA62064A32F810009D
:104170000882A1F86000A1F862007047F0010020F9
:10418000E2B80008D6B800082DE9F05FFB48FC490A
:1041900082880B889A1A92B20F2A47D309888180A5
:1041A000F8498346F84D0888F84FDFF8E4934FF05C
:1041B0000108002678B3401E0880EE73EE624A467E
:1041C0002868B2F90220430742F6AA2118D4FB88D6
:1041D00043F40053FB8099F800309B0709D5AB6886
:1041E00023F08003AB60A5F8806085F8826085F8D5
:1041F0008360C30404D485F8F480C5F8F06003E05C
:1042000085F8F460430707D48A4205DB85F8F88017
:10421000A5F8F66004E010E085F8F860430703D4E1
:104220008A4201DBC00703D085F81561BDE8F09F25
:1042300085F81581A5F81661F8E7B5F81C0143F675
:104240009821884202D2401CA5F81C0102F072FAA3
:10425000DFF840A39AF8500010B1FEF719F905E015
:10426000C6481838017821F001010170FFF71AFBE8
:1042700000F028FAC84841F26802416C4FF400602F
:10428000914201DBC54A04E0B1F57A6F02DAC34A14
:10429000121D1060BF48DFF8F0A20A2490F8510008
:1042A000AAF1340AC00738D0BD48807B802802D3E9
:1042B0002878800705D5BB480078C20601D480065F
:1042C00027D5EA7B8AF8072099F80030AB4A23F01B
:1042D0000203183A89F8003056801378504623F0CC
:1042E00001031370BA7952060FD48289B2F5FA7FAE
:1042F00003D2521CAAF80C200FE040F63C70814219
:1043000001DD002465E0042463E00024AAF80C60C9
:104310005FE08AF80360AAF80C60A868020501D57E
:10432000082456E09B4A92F83FE05FEACE7245D0FF
:104330009B4BEA7B8AF807205B7A802B43D39A4B0E
:104340009B781B063FD52B785B0730D4FB889B04FA
:1043500004D500BF20F02000A8602FE0874B40F07C
:104360002000183B5E801C7824F001041C70A860BB
:104370008B48C37D802B0AD303F07F0400684FF085
:104380000043E340184202D185F8048000E02E711A
:104390002879C00702D15FEA8E7005D50324032A6D
:1043A00017D08AF80A8014E00024EE6211E020F0B1
:1043B0002000A860F88820F40050F88095F82A01C1
:1043C000012805D005E02A6842F004022A60C1E70E
:1043D000092408B2754903F065FB6B49744DCA6A3C
:1043E00050438013A1F8E8000A2C6FD16E48807802
:1043F000800602D5FCF73CFD09E063488168CA05E8
:1044000002D521F0080101E041F0080181605E4819
:104410004FF40054620090F84A8042F6CC4142F2D8
:104420006663B8F1010F1FD0B8F1020F31D0DFF889
:1044300084C12978B8F1030F3ED0C1F38108911EE1
:10444000B8F1010F3FD0B8F1020F3CD0A0F818210D
:10445000A0F8482047F23C31ACF800104D4991F8E3
:104460007010012933D03FE095F800C0CCF3810CE7
:10447000BCF1010F07D0BCF1020F07D0A0F8181152
:10448000A0F84810EAE7A0F81831F9E7A0F81841B9
:10449000F6E795F800C0CCF3810CBCF1010F08D011
:1044A000BCF1020F05D0A0F8182100BFA0F84820E9
:1044B000D4E7A0F81811F9E7A0F81821A0F84820CF
:1044C00046F65471C8E7A0F81811C1E77BE02978D7
:1044D000C1F3810101290ED002290FD041F6E1215B
:1044E000A0F81811A0F84830244918390B78DB07D8
:1044F00007D00B8A07E0A0F81831F3E7A0F81841BD
:10450000F0E7B9F80430ABF8123019B2B0F948301E
:104510005943C1F38F335146AAF81830934200D95A
:104520000A83254A1278D20605D50B8B41F2333225
:10453000934200D20A838268C2F3C003C2F300240C
:10454000A34205D10C8B41F699139C4200D90B83F1
:104550001A4B9B78DB0707D0D20105D4114A127899
:1045600002F00F02032A00D00E83BAF81810C162BD
:10457000002927DD12480224067024E0C80A002022
:10458000480700204A070020A4020020000C002059
:10459000E2050020580E002038010020100C0140D8
:1045A000E8050020AF0700208F070020DCAE0008E0
:1045B000D004002030010020100700207F070020D9
:1045C0005C07002000249BF81A0028BB022C15D0A1
:1045D00014B323490878830608D5BB795B0605D553
:1045E000204B1B78DB0963F386100870F88820F4F1
:1045F0000060F880B9F8041039B109E0288F00286C
:10460000E7D143F698202887E3E720F08000F88080
:1046100080B220F02000F8801148406C4E2819DB51
:10462000F888010616D5BAF816305B1C9BB2AAF8BA
:104630001630B3F5FA6F07D3AAF81660B9F804106C
:1046400011B920F08000F88099F8001021F00201E3
:1046500089F8001004488BF81A40C473E6E500009E
:104660003801002010070020A402002070B50023AC
:104670000C8863F30F02012505FA03F6344206D0D5
:10468000C3F10F0605FA06F1114361F30F025B1C3B
:10469000102BF1DB028070BD70B500230C7863F342
:1046A0000702012505FA03F6344206D0C3F10706D6
:1046B00005FA06F1114361F307025B1C082BF1DBDD
:1046C000027070BDF0B5204890F866101F480129AF
:1046D000836823F4006234D11D49CE88740630D437
:1046E0001C4D1F054FF00004B5F9025020D41A4AA2
:1046F000526C642A11DC40F6386295420DDAB2043D
:104700000BD40278520710D4B0F8D82040F6B83550
:10471000AA4203D2521CA0F8D820F0BD43F4006294
:104720008260D001F9D44C81F0BDA0F8D840F0BD32
:1047300041F2CD039D42FADD897AC907F7D1826043
:10474000F3E78260F0BD0000580E0020A4020020B4
:10475000000C0020E205002038010020F0B5364DA5
:10476000364F044695F83B0097F83B1023780843F2
:10477000EE1C6278834205D1E0781146FEF7DCFE3C
:10478000207908E094F802C084450CD1E178104605
:10479000FEF7D2FEE07905F82F0F2878805D68706B
:1047A000287BE877F0BD82421DD161461846FEF7AE
:1047B000C3FE95F84E1095F83B00814207D1B97AB7
:1047C00009B1A17900E0617985F82F101EE06978C0
:1047D000012901D0A17922E0617927E0297841F00F
:1047E0000401297012E0E1788142DBD1194660466C
:1047F000FEF7A2FE95F84E1095F83B0081420AD1D3
:10480000B97A09B1617ADFE7217ADDE715F82F1F60
:10481000895D6970C5E76978012906D0617A85F8F4
:104820002F10B97A0029F1D1D8E7217A85F82F1015
:10483000B97A0029EAD0D1E75804002038010020D5
:104840000B48017821F0020100F8381B002100F824
:104850001819417781773321818541850821418469
:10486000012100F81F1C034880F839107047000030
:1048700058040020380100200D4900B50B4851F8BC
:10488000012F40F8032F89888180084801210930D1
:10489000FEF780FF054802211330FEF77BFF034837
:1048A00004211D305DF804EBFEF774BF58040020AE
:1048B00038010020094944F648000880091D46F6E1
:1048C00048000880091D41F2111008800348001FAC
:1048D000018841F02001018070470000182C014040
:1048E0002DE9F047664C674B0025A0780126654A04
:1048F000103305287ED2DFE800F00313113E1100CB
:10490000108820F0010010801D805F480580001F86
:104910000580001F0580FFF7CDFFA670BDE8F0877A
:10492000594941F6CC401C390880574945F6580092
:1049300024390880091D46F6580008805249202075
:10494000283908800020401CC0B27328FBD3FFF731
:10495000B1FF4C4984F85C502C3147F690600880D8
:104960004848143006801D80108840F001001080F7
:104970000220A070D2E700215FF0010004EB4102A9
:1049800004EB4003B2F85020B3F850309A4200D202
:104990000146401CC0B20628F0D33C48405C84F875
:1049A0003900FFF74DFF1D2000F0B8FD00F076F84C
:1049B000374E38484FF4807996F83B10012904D0DF
:1049C00002291BD0042930D047E040218046FEF761
:1049D0006FFE870080214046FEF76AFE47EA4007E7
:1049E00049464046FEF764FE074347F0010084F85D
:1049F0003B0000E03DE0224809302CE040218046A9
:104A0000FEF756FE870080214046FEF751FE47EA3A
:104A1000400749464046FEF74BFE074347F0020079
:104A200084F83B001648133015E040218046FEF71D
:104A30003FFE870080214046FEF73AFE47EA4007E6
:104A400049464046FEF734FE074347F0040084F829
:104A50003B000B481D3003F021FB94F82F0086F833
:104A600038001D2000F070FD0420A0700A48057079
:104A700054E7108820F0010010801D80A5704DE7DC
:104A800058040020000800403C2C014098AF00086A
:104A900038010020001001403F0700202DE9F041BF
:104AA000344C14F82F0F344DE07240212846FEF7A5
:104AB000FFFD860080212846FEF7FAFD46EA400603
:104AC000AF1539462846FEF7F3FD0643207BF1B2C9
:104AD0002F3C814215D084F83C0040212846FEF747
:104AE000E7FD860080212846FEF7E2FD46EA400603
:104AF00039462846FEF7DCFD064384F83B60FEF7A6
:104B0000EFFF1E4D95F83B00012827D0022828D042
:104B1000042829D0174894F83B102730085C04F883
:104B2000300F14F80109FEF76DFE04F82F09A87A7A
:104B300000B10120607001F0A5FE94F84E0094F8D9
:104B40003B10884206D094F83800062802D2401C58
:104B500084F8380084F84E10BDE8F081054809302B
:104B600004E00448133001E002481D30BDE8F04184
:104B7000FFF7F4BD58040020001001403801002068
:104B8000FF2801D9FF207047C0B270472DE9F041DE
:104B90004A4991F87200AA2874D191F873005528F7
:104BA00070D1474C00200A5C2254401CC0B27428CB
:104BB000F9D3444E2069C6F80100A08AA6F8050082
:104BC000D4F81600F060D4F81A003061D4F81E0052
:104BD0001234706103F008FA3B49608A888103F05F
:104BE0001DFA207D123CC007307802D040F004004E
:104BF00001E020F00400354930704FF48040086136
:104C0000334D14F8280F334985F82000608B6880F5
:104C1000A08BA880E08BE880208C2881608C688144
:104C200094F8240081F8D60014F8010C86F83B00B3
:104C30000027C6F89C70FFF71FFE2748A18E01834E
:104C4000E18E4183218F818394F84210283C012911
:104C500008D0022901D0032909D0297821F00C01BC
:104C6000083107E0297821F00C01091D02E02978BC
:104C700041F00C01297094F8642018491AB10122FE
:104C80004A8101E00EE04F8194F8701001290BD0A9
:104C900094F86D1059B101290CD04FF4805100BF28
:104CA000A0F87610BDE8F08144F21C71F8E74FF4EB
:104CB0000051F5E741F25551F2E7000000FC000811
:104CC000580E0020380100204C000020F80D002074
:104CD000D0040020A402002038050020000C002091
:104CE00010B5FCF7D1FCFE48FE4AFF49807AC007A8
:104CF00003D0887820F0010005E09078800703D089
:104D0000887840F001008870F8480B7803704B7881
:104D100043708B788370CB78C3700B7903714B79B8
:104D200043718B798371C979C171EF490831097871
:104D30000172ED49083149784172EB4908318978AF
:104D40008172E9490831C978C172E74908310979A6
:104D50000173E549083149794173E349083189799B
:104D60008173E1490831C979C173DF49103109788C
:104D70000174DD49103149784174DB49103189787B
:104D80008174D9491031C978C174D7491031097972
:104D90000175D549103149794175D3491031897967
:104DA0008175D1491031C979C175CF4918310B7856
:104DB00003764B7843768B788376CB78C3760B7902
:104DC00003774B7943778B798377C979C177C64964
:104DD0000F39097880F82010C3490F39497880F8D5
:104DE0002110C1490F39897880F82210BE490F3946
:104DF000C97880F82310BC490F39097980F824104C
:104E0000B9490F39497980F82510B7490F3989799F
:104E100080F82610B44920310B7880F828304B7880
:104E200080F829308B7880F82A30CB7880F82B30C6
:104E30000B7980F82C304B7980F82D308B7980F805
:104E40002E30C97980F82F1000F1D001097880F850
:104E5000301000F1D001497880F8311000F1D00114
:104E6000897880F8321000F1D001C97880F83310C9
:104E700000F1D001097980F8341000F1D0014979AE
:104E800080F8351000F1D001897980F8361000F1F2
:104E9000D001C97980F8371000F1D001097A80F883
:104EA000381000F1D001497A80F8391000F1D001B2
:104EB000897A80F83A1000F1D001C97A80F83B1065
:104EC00000F1D001097B80F83C1000F1D001497B52
:104ED00080F83D1000F1D001897B80F83E1000F190
:104EE000D001C97B80F83F1000F1D001097C80F827
:104EF000401000F1D001497C80F8411000F1D00150
:104F0000897C80F8421000F1D001C97C80F8431000
:104F100000F1D001097D80F8441000F1D001497DF5
:104F200080F8451000F1D001897D80F8461000F12D
:104F3000D001C97D80F8471000F1D001097E80F8CA
:104F4000481000F1D001497E80F8491000F1D001ED
:104F5000897E80F84A1000F1D001C97E80F84B109C
:104F600000F1D001097F80F84C1000F1D001497F99
:104F700080F84D1000F1D001897F80F84E1000F1CB
:104F8000D001C97F80F84F1000F1F0010B7880F854
:104F900050304B7880F851308B7880F85230CB7895
:104FA00080F853300B7980F854304B7980F85530C5
:104FB0008B7980F85630CB7980F857300B7A80F8AF
:104FC00058304B7A80F859308B7A80F85A30CB7A47
:104FD00080F85B300B7B80F85C304B7B80F85D3079
:104FE0008B7B80F85E30CB7B80F85F300B7C80F869
:104FF00060304B7C80F861308B7C80F86230CB7CF9
:1050000080F863300B7D80F864304B7D80F865302C
:105010008B7D80F86630CB7D80F867300B7E80F822
:1050200068304B7E80F869308B7E80F86A30CB7EAA
:1050300080F86B300B7F80F86C304B7F80F86D30E0
:105040008B7F80F86E30C97F80F86F102649503111
:105050000B7880F870304B7880F871308B7880F85E
:105060007230CB7880F873300B7980F874304B79DC
:1050700080F875308B7980F87630C97980F87710B0
:10508000117880F88010517880F88110917801F0C3
:10509000030180F88210117980F88310517980F82B
:1050A0008410917980F88510D17980F88610117A72
:1050B00080F887100C4938310A7802F0030280F832
:1050C00088204A7880F889208A7880F88A20CA78EF
:1050D00080F88B200A7980F88C204A7908E000005B
:1050E000000C0020101000207F070020000F00207F
:1050F00080F88D208A7980F88E20C97980F88F1009
:105100006B490A7880F890204A7880F891208A7854
:1051100080F89220CA7880F893200A7980F8942049
:105120004A7980F895208A7980F89620C97980F8A4
:1051300097105F4908310A7880F898204A7880F8FB
:1051400099208A7880F89A20CA7880F89B200A797A
:1051500080F89C204A7980F89D208A7980F89E20EA
:10516000C97980F89F10524918310A7880F8A02038
:105170004A7880F8A1208A7880F8A220CA7880F83E
:10518000A3200A7980F8A4204A79C2F3400363F38C
:105190005F0280F8A5208A7980F8A620C97980F876
:1051A000A710434920310A7802F0010280F8A820B4
:1051B0004A7880F8A9208A7880F8AA20CA7880F8EE
:1051C000AB200A7980F8AC204A7980F8AD208A7942
:1051D00080F8AE20C97980F8AF10354928310A78B7
:1051E00080F8B0204A7880F8B1208A7802F0030273
:1051F00080F8B220CA7880F8B3200A7980F8B42009
:105200004A7980F8B5208A7980F8B620C97980F883
:10521000B710274930310A7880F8B8204A7880F8EA
:10522000B9208A7880F8BA20CA7880F8BB200A7939
:1052300080F8BC204A7980F8BD208A7980F8BE20A9
:10524000C97980F8BF101A4938310A7880F8C0202F
:105250004A7880F8C1208A7880F8C220CA7880F81D
:10526000C3200A7980F8C4204A7980F8C5208A7959
:1052700080F8C620C97980F8C7100D4940310A78F6
:1052800080F8C8204A7880F8C9208A7880F8CA2037
:10529000CA7880F8CB200A7980F8CC204A7980F847
:1052A000CD208A7980F8CE20C97980F8CF1010BD42
:1052B000BF0700207CB50121082000F08BFC4FF4D3
:1052C0000050ADF8040010248DF8074001208DF83F
:1052D000060001A91548FEF76DF90121092000F02B
:1052E00079FC01211248FEF7B7F90820ADF800005B
:1052F00004208DF803000F4E03258DF802506946F7
:105300003046FEF757F908213046FEF7D8F9ADF8D8
:1053100000408DF803408DF8025069463046FEF794
:1053200049F910213046FEF7CAF97CBD001401404E
:1053300000023000000C0140FEE7000038B50121FA
:10534000082000F047FC4FF44060ADF80000482012
:105350008DF8030003201B4D8DF802006946284696
:10536000FEF728F929152846FEF7A2F9164CE9148C
:10537000607020702846FEF79BF9E070A070FEF781
:10538000BFF9A080E080114890F84A10104849B158
:1053900001290BD002290FD003290CD1C17841F08B
:1053A000030107E0C17821F0030103E0C17821F097
:1053B0000301491CC17038BDC17821F00301891C6B
:1053C000F8E70000000C014080080020A402002043
:1053D0007F0700202DE9F041444D4FF480612846BD
:1053E000FEF766F90446E9142846FEF761F9DFF88E
:1053F00000810746002598F800002E46844205D01B
:1054000088F80040FEF77CF9A8F8040098F801003D
:10541000844209D0B8F80400FEF75AF91E2803D3D5
:1054200088F80140A4B3002598F80200444687425A
:1054300003D0A770FEF764F9E080E078874207D0D8
:10544000E088FEF745F91E2802D3E7701FB3002657
:1054500060782849002808791FD020F002000871E0
:10546000E278EAB120F0010008710DB1002E37D1C9
:1054700055EA060034D0204BDA7802F00300032806
:1054800000D90320002475B103280CD2401C1AE077
:10549000FFE70125C8E70126DAE740F00200DEE772
:1054A00040F00100E0E776B168B1012809D1134D61
:1054B0006D6CB5F5FA6F04DA8978C90603D500205A
:1054C00001E0401EC0B260F301020D49DA7048B13C
:1054D000012803D0022801D0032801D181F84A0015
:1054E000BDE8F08181F84A40FAE70000000C014075
:1054F000800800208F0700207F070020380100204F
:10550000A4020020704700F01F02012191404009D1
:10551000800000F1E020C0F88011704700F01F0209
:10552000012191404009800000F1E020C0F8801185
:10553000704700F01F02012191404009800000F1F6
:10554000E020C0F80011704700F01F0201219140D7
:105550004009800000F1E020C0F800117047000011
:1055600070B50F23C47801780122F4B1144C24687B
:10557000457804F4E064C4F5E064240AC4F1040648
:10558000E3408478B5401C402C4301F1E021230125
:1055900081F80034007800F01F018A404009800043
:1055A00000F1E020C0F8002170BD01F01F00824032
:1055B0004809800000F1E020C0F8802170BD0000A3
:1055C0000CED00E002490843024908607047000002
:1055D0000000FA050CED00E02DE9F05F00261D202B
:1055E000FFF791FF6C4CDFF8B4B1A4F1B800A77ECF
:1055F00090F83810DFF8A8E1DFF8A8A100258F4265
:105600007ED0E776A176626A036B5A434FEA12496D
:105610009BF80820120702D51EF8012000E00A4678
:1056200094F812C0BCF1010F09D004EB4206B6F9A0
:1056300002C0C4F828C0B6F90460E6620CE043F684
:10564000FF7CC4E90A5C90F83DC05FEACC7C01D0E5
:1056500012B102E0052A00D1012600EB47074FF006
:10566000804CBF893F04B7FBF3F3E361476BBCFB9E
:10567000F7F7276294F813C0BCF1000F06D0BCF115
:10568000010F05D03B4403EBD3735B10636201E071
:105690003B466762DFF810C14FF6FF7707EA8307E2
:1056A000ACF808709AF8007090F80A8090F83DC045
:1056B000082F08F003070CF0030C05D067450BD149
:1056C000B8F1000F05D008E0674505D0B8F1000F2C
:1056D00003D05B42636200E06562C6B1636A002B7F
:1056E00003D006DD228D05E00AE0304B33F81220AE
:1056F00000E0A28DA4F86020227822F0200222701F
:105700009AF80020042A07D0082A05D012E0B4F83D
:10571000603003EB0902EDE780F8405065629BF8CA
:105720000800000701D51EF80110204830F81100CC
:10573000A4F860001E49606A09883E314843B4F805
:10574000601001EB204006B21D20FFF7F2FE606AF8
:10575000002807D021784FEA81600ADD002804DAAA
:10576000A08D09E0B4F8600006E0E06AB04208DB12
:105770000CE0002802DA208D208208E0A06AB04206
:1057800004DD208241F02000207000E02682257593
:1057900065752586BDE8F09FF0010020A402002079
:1057A000C4B800083F070020940B0020D6B80008BA
:1057B0002404004043184FF48042934210DD90428D
:1057C00002DD104600210BE0914202DD002011466F
:1057D00006E08003B0FBF3F000B2C0F5804109B2EF
:1057E00041EA00407047F0B541F2F1130022C36076
:1057F0000E24826204824BF2660508264561068308
:1058000043F6FF774283878340F2492E4FEA873C75
:10581000C0F808E0C0E9082CCB608A620C824D61B8
:105820000E834A838F83B4208860C1E9082CF0BDC1
:10583000002181620949C1600E210182084941614C
:10584000082101834FF44041418343F6FF71818376
:10585000090701620349416270470000B6A00100D8
:105860001C0C010000C0FF0F064941F68160088052
:1058700005480168054A01F4E06111430160BFF386
:105880004F8FFEE7442C01400CED00E00400FA05C8
:10589000F8B501210D2000F09DF94FF4E060ADF85E
:1058A000000018241D4E8DF8034003258DF802508A
:1058B00069463046FDF77EFEB1153046FDF7FFFE26
:1058C00071153046FDF7FBFE31153046FDF7F7FE4A
:1058D0004FF46040ADF800008DF80340104C8DF897
:1058E000025069462046FDF765FE61142046FDF72B
:1058F000E8FE4FF480412046FDF7E3FE4FF40041FF
:105900002046FDF7DEFEA014ADF8000048208DF81B
:10591000030069462046FDF74DFEF8BD0008014032
:10592000000C01402DE9F0410121CE028CB030463F
:1059300000F050F9DFF87081404601F033FC08A810
:1059400001F05CFE4FF45860ADF824000024ADF87F
:1059500020402020ADF822000125ADF826408DF82A
:10596000285008A9404601F0FBFD0021404601F007
:105970004EFE4FF6FF71404601F053FE012200211A
:10598000404601F0DFFD0121404601F0C7FB04A8BD
:1059900001F0DFFBADF81060A802ADF81200ADF821
:1059A00014408120ADF816002803ADF81800ADF8BA
:1059B0001A40ADF81C4004A9404601F0B9FBADF80F
:1059C00008400820ADF80A006027ADF80C408001BF
:1059D000ADF80070ADF80440ADF80E00ADF802402F
:1059E000ADF806406946404601F09CFC69464046D9
:1059F00001F0DEFC6946404601F024FDADF804509C
:105A000040F61450ADF80070ADF80600ADF808404F
:105A1000ADF80C40ADF80250ADF80A40ADF80E40BC
:105A20006946404601F052FD0121404601F09AFBD3
:105A30000821404601F0B6FC3146404601F0F8FC32
:105A40000821404601F03CFD3146404601F070FD22
:105A50007021404601F079FD18208DF82C008DF85A
:105A60002D408DF82E408DF82F500BA8FFF778FDB4
:105A70000D480C30018841F0800101800A48143043
:105A8000018841F001010180001F0480012140468E
:105A900001F072FB8DF828500121404601F076FBA1
:105AA0000CB0BDE8F0810000002C0140704740F2CE
:105AB00013414160082181608621C1604FF480411B
:105AC00001614942416100210162C1627047016286
:105AD0007047000010B501884288891A09B2018315
:105AE000B1F5005F02DBA1F5804104E011F5005F34
:105AF00002DC01F580410183B0F91820416851436F
:105B0000C1618368846A5343C2681B12624303EB1A
:105B10002222036A1A44114402628A1342624169D2
:105B20008A4203DB01698A4200DC11468A1AC0E915
:105B30000A21028E4FF40373594302EBA13202860D
:105B40000B4A1278082A04D10A4A936F03EBA13159
:105B50009167B0F93010B1F5804F02DDA1F58041B9
:105B600003E0002902DA01F58041018610BD000042
:105B70003F070020140C0020034A516821F44041E3
:105B8000014351607047000000100240044A0029A0
:105B9000516901D0014300E0814351617047000029
:105BA00000100240044A0029D16901D0014300E0FD
:105BB0008143D1617047000000100240044A00296F
:105BC000116901D0014300E0814311617047000079
:105BD00000100240044A0029916901D0014300E00D
:105BE000814391617047000000100240044A00297F
:105BF000D16801D0014300E08143D16070470000CB
:105C0000001002402DE9F041274CA6154021204606
:105C1000FDF74EFD850080212046FDF749FD45EA50
:105C2000400531462046FDF743FD0543EDB24021D6
:105C30002046FDF73DFD870080212046FDF738FD19
:105C400047EA400731462046FDF732FD0743F8B2E8
:105C5000A842DBD140212046FDF72AFD87008021A4
:105C60002046FDF725FD47EA400731462046FDF76F
:105C70001FFD0743F8B2A842C8D140212046FDF7D6
:105C800017FD870080212046FDF712FD47EA4007F7
:105C900031462046FDF70CFD0743F8B2A842B5D1C6
:105CA0002846BDE8F08100000010014010B50268F0
:105CB000416802FB02F301FB0133B3F1805F11D9AC
:105CC0001B0E103B0A4C9BB212B234F8133009B2CF
:105CD0005A43594342F38F3241F38F31C0E90221D5
:105CE000012102E0C0E902210021017410BD000081
:105CF000B0AE00082DE9F05FFB48FC4902880B8834
:105D00009A1A92B20F2A7DD309880180F848024678
:105D10008189D2884B0703D48B0701D4CB0702D0EB
:105D200042F4007201E022F40072C2808246080749
:105D300002D45046C90604D5BAF8061041F0010154
:105D400002E0C18821F00101AAF80610E848FDF739
:105D500057FAE848B0F93A10B1F5804F02DA491C19
:105D6000418703E0E3494FF480404887DFF8889398
:105D700041F6CC40E149D9F85020824203DD8868E1
:105D800020F010008860DE4BDE4E0024188820B121
:105D9000401E1880CC73347029E0BAF80600450420
:105DA0001DD4BAF80C30DD0619D41D0717D405062A
:105DB00015D4850613D4050511D4450603D5D24D57
:105DC0002D782D060BD5450709D4C50507D4050741
:105DD00005D4850403D4C00601D4D80707D0CB4826
:105DE000CC73CB4B3470C4831C8080F828408B4626
:105DF000B1F84210DFF81C83C74869B1491EABF8FF
:105E0000421000E0E6E098F8005025F0020588F81E
:105E100000508BF80F400BE098F8003043F002037D
:105E200088F800303178012903D10178062900D1A2
:105E300034703178DFF8E4E2B94D01270A2973D2D2
:105E4000DFE801F0FDC805C8FCFBC872FAF902F0F2
:105E5000E1F9DFF8A8A2A849AAF1340A40F62822FD
:105E6000BAF81C00401C80B2AAF81C00496C914290
:105E700002DAAAF81C4013E09E4A40F6CC43D268EE
:105E80009A420DDBB8F9042043F699139A4207DBD6
:105E9000B0F5FA7F04D3287810B9AAF81C402F7007
:105EA000A04A108868B19AF804305B1CDBB28AF80B
:105EB0000430022B05D39C488AF8044003885B1CFD
:105EC00003809BF80F00D846092814D002287CD004
:105ED000A8F83441B8F84400DFF850B2A146C8B180
:105EE00041F288344846AAF81C90A14221DA297868
:105EF00001291AD01DE07C484430FDF72BFDFDF749
:105F0000F5F97D48416CCAF8301041F27C51CAF86D
:105F1000201089E2A88AA8F83400E86A6863A86AB1
:105F20002863A8F844703BE0C0E17F4928700880EE
:105F3000108098F84A10022908D09BF80310B7EB9C
:105F4000511F10D098F82C1151B104E098F82C1181
:105F500009B96FF0A200C8F8DC0088F8EE7008E01C
:105F60006FF40560F7E7C8F8DC0088F8EE00CAF8BF
:105F700028009BF80300B8F93410B7EB501F07D086
:105F8000B8F8DC004FF42F7300B240F2DC5203E0AB
:105F90004FF47A735A00002000F0C2FBA8F83400D6
:105FA0009BF803106248B7EB511F53494FF49A73A3
:105FB000496C11D0B1F5FA7F0CDAB5F90A109942A3
:105FC00008DC00BF86F8009000E020E088F8EE9042
:105FD000A0F81A90BDE8F09F40F2DC52914203DA3B
:105FE000B5F90A209A42EDDDB8F8442040F6C41312
:105FF000521C92B2A8F844209A42E3D23D4AD26899
:10600000002AE7DC42F6E0629142DBDAE2E7B8F828
:10601000340140F6B832904207D2334B183B1B781C
:10602000DB0702D1401CA8F8340183B240F2DC50F7
:10603000834208D804E0CEE0ACE0F3E0EEE0F6E026
:1060400042F6CC4003E0A8F8342143F26660E867EA
:10605000CAF830108AF80970364EA8F8444088F81B
:10606000EE40707F5546F8B1F07FE0B3B8F82C00F1
:10607000B8F9341000B20A23052200F051FBA8F849
:106080003400F47786F81D40B8F91A01B8F91811F0
:1060900088426ADA697901F1010111F0FF01697141
:1060A0006AD06C71401C62E04FF48040A8F8E800B0
:1060B000D8F82C10814200DA08461F4900B26883E4
:1060C00091F84D1051B998F84A203AB1B8F8081033
:1060D000C1F3C003C1F300218B422FD13623B8F99D
:1060E0003410052234E03CE0C80A002048070020B4
:1060F000000C00203805002038010020A4020020F8
:106100004C0700203F07002010070020300A002025
:1061100006000020E2050020400700205802002071
:106120004C000020080000200A000020A7070020E3
:106130003C0B0020200E0020580E0020012A03D026
:10614000022A01D0032A06D0B8F93410DA23242217
:1061500000F0E6FA06E0B8F9341040F29913512243
:10616000F6E7A320A8F834008EE703DD801EA8F828
:106170001A0101E0A8F81A11B8F934004FF480416F
:10618000884202DDA8F8341024E70028FCDAA8F8D9
:1061900034401FE7D84ADBF8E0105846914202D25B
:1061A000491CC0F8E010C17B082903D1D0F8E010E9
:1061B00091420CD334708168CA0502D521F00801E0
:1061C00001E041F008018160CBF8E04002E7BDE862
:1061D000F05F02F09DBF9BF80F005F46092803D0D7
:1061E000BC868BF80F4061E1C44D686A401C686250
:1061F000022809DD288E012301B2288C052200B275
:1062000000F08EFA6C622863BD48298E0180B9F8CF
:1062100044104180FDF7B6FBB886DBE6BDE8F05FD1
:1062200004F0E6BC9EF8000009287DD0D2E68BF889
:1062300011419BF82C3163B142F31101CBF8DC40E2
:10624000B04A8B03E962891093628A03A962AE495E
:106250008A62AA498C83D9F8442041F288318A4263
:1062600007DA2978012904D1A8492C700C80A849A3
:106270000C80A84ADFF8A0C21188491C8BB2A7493C
:106280001380C82B04D391F80080B8F1010F19D006
:10629000B3F57A7F04D391F80080B8F1020F11D0E2
:1062A000B3F5FA6F02D30B78032B0BD09BF80F10CA
:1062B000891E08297ED2DFE801F010B9FBF7047DC2
:1062C00085AB87E60C701480BAF8062022F40062D1
:1062D000AAF806208CF80070E8E7D9F84410C84600
:1062E000822904DA0178062901D00470F5E0FDF76F
:1062F00037FA98F80000400613D5894880780428BA
:106300000FD0D8F84410404682290ADA817A98F8EA
:106310003D0001F0030100F00300814201D001F0D3
:1063200029FEB146307800E0C0E00628C9D088F8E0
:106330003F40D8F85000734940F311008203E862EF
:1063400080108A628103A8626F4846468162FCF72A
:10635000CDFF6A485D464772BBF81801ABF81A01D9
:10636000706CABF88640B0F5437F10DD4FF4804091
:10637000A5F88400A86840F48060A86096F83810FA
:1063800005299ED140F01000CBF8080016E04FF42C
:106390008041A5F88410A96821F48061A96040F2C9
:1063A0008A21884204DA3078400601D402F09EFD4A
:1063B000A86800E098E040F01000A860022089F88A
:1063C000000007E6D9F84410B1F5437F02DA0178FE
:1063D00006298AD15348017821F040010170FCF769
:1063E00085FF43F6FE70ABF81A010BF1E005FDF7EF
:1063F000B7F94D4810F8341F21F0010101704249EE
:106400002C608C623F498C62082131704464E1E564
:106410003B48FDF79FFAFCF769FF3848D9F844106C
:10642000016341F27C51016209203BE09AF80600C9
:10643000C006C6D4D9F844004D46B0F57A7F35DDA4
:10644000FDF78EF92878400611D535488078042864
:106450000DD0686C82280ADAA87A95F83D1000F011
:10646000030001F00301884201D001F083FD85F8AB
:106470003F40B5F85000ABF8340001B24FF4804013
:106480005C46814200DDA086FCF730FFA06840F446
:106490008060A06095F83810052992D140F0100076
:1064A000A0600220307095E514E001E0347091E5C1
:1064B000D9F84410B1F5437F02DA0178062988D172
:1064C000BAF8061021F02001AAF80610FDF748F9E5
:1064D0000420E7E70078062801D037707AE5092024
:1064E0008EF800000520DDE70D498C70047085F8FA
:1064F0005E40ABF834406DE5C0D40100700200206E
:106500000C0B0020000A0020D00900200A00002007
:1065100008000020100100200E01002012010020C0
:10652000580400204E070020140C002030B585B020
:1065300001210420FFF74EFB4FF40040ADF810009E
:1065400048208DF8130004A91848FDF733F80121FD
:106550000846FFF727FB40F68C20ADF80400032423
:106560000020ADF80040ADF80200ADF806004FF095
:1065700080456946284600F0F3FF1C208DF80C008A
:106580008DF80D408DF80E4001208DF80F0003A806
:10659000FEF7E6FF01221146284600F0BBFE01216E
:1065A000284600F0E9FD05B030BD000000080140BC
:1065B000704700002DE9F041304CE07800285AD1B6
:1065C0002078002857D0401E10F0FF00207052D1D4
:1065D0004FF49670208272B6294F45F2AA50A7F860
:1065E00072000020FCF760FE264D13202860FCF7A7
:1065F0006DFEA8BB3420E86002202861224E6E6147
:10660000286940F040002861FCF760FE40BB002193
:106610001E4A08465FEA255312F800C0BCF1FF0F7E
:1066200000D00121401C80B29842F5D3C1B9C4E921
:10663000067639260127A06910F8011B10F8012BF6
:10664000A061E06901EB022102886A612F6120F8F4
:10665000021BE061FCF73AFE10B9761EB6B2EAD230
:106660000120FCF721FE62B601F0D8FC08488168E1
:1066700021F480418160BDE8F08100003C070020EA
:10668000580E00200020024000FC000800FC00081A
:10669000A40200201948016841F01001016001685E
:1066A00021F003010160016841F00201016014481A
:1066B0004168416041684160416841F480614160E6
:1066C000416821F47C11416041680E4A11434160E8
:1066D000016841F08071016001688901FCD5416861
:1066E00021F003014160416841F0020141604168CD
:1066F000C1F381010229FAD1704700000020024055
:10670000001002400000280830B5044C039D608052
:10671000A180E2802381658130BD0000F40B002060
:106720000A44824201DA10B27047C91A8142FBDD85
:1067300008B270472DE9F04F4A48DFF82CA1DFF886
:106740002CB1C17F477A046849480022DFF82C91B8
:10675000466C48484FF0010E80298578464883688A
:1067600034D301F01F0C5AF82C100C420146096872
:1067700002D041F4805101E021F4805101605FEAD0
:10678000C14C1ED45FEA814C1BD599F80AC0C8469B
:106790005FEACC7C0BD05FEAC31C12D4A8F80A20B5
:1067A0009BF8008028F002088BF8008009E0322E68
:1067B00007DC5FEA857C04D55FEA035C01D4A8F8B6
:1067C0000AE04FEA113C6CF34D310160802F24D375
:1067D00007F01F075AF827100C42016802D041F059
:1067E000040101E021F0040101604C0711D44C05C3
:1067F0000FD599F80A70FF070BD0DF0109D4A9F86B
:106800000A209BF8007027F002078BF80070C0F890
:106810009C208C0864F38A21016099F80A40E407FF
:1068200019D1174C94F86440012C14D1322E10DC8D
:10683000046866070DD51B050BD4E30409D5AB0727
:1068400007D5D0F89C304EF66024A34205D9A9F8AC
:106850000AE0C0F89C20BDE8F08F5B1CC0F89C30BB
:10686000F9E70000E805002000B40008E205002078
:10687000380100208F070020A4020020000C002017
:10688000580E002010B5FAF789FA0F48018821F058
:10689000020101800C49183109880C4A928E11447A
:1068A000094A3432118008490C390A8842F0010241
:1068B0000A80011D0A884FF6ED531A400A800188AC
:1068C00041F01201018010BD0C040040580400206A
:1068D000130A03700A70704705484FF6FF6201887B
:1068E000491C89B20180914201D300210180704787
:1068F000880800200F4810B5016841F001010160CF
:1069000041680D4A1140416001680C4A1140016024
:10691000016821F480210160416821F4FE01416099
:106920004FF41F018160FFF7B5FE05494FF000608D
:10693000086010BD001002400000FFF8FFFFF6FEE7
:1069400008ED00E04FF0E02005494161054AF021E3
:1069500082F8141D00218161072101617047000048
:10696000DFA501000FE000E02DE9F047DFF8D4A03B
:10697000BAF800004FF00005000635D5324C6088AB
:10698000401C6080FBF75AFDDFF8C0C0304A314838
:106990009CF80070677092F800800723C8262E4983
:1069A0004FF00509B8F1010F22D02C4FB7F806C0FF
:1069B000BCF1000F38D084F80090848944F00804BA
:1069C0008481C48824F40064C480886820F00400B2
:1069D0008860FD801370A1F8426000204FF496613A
:1069E000401C80B28842FBD3AAF80050BDE8F08773
:1069F00077B1012F12D0C78847F40067C780886835
:106A000040F004008860032020708CF80090E1E7DB
:106A1000878947F0080787810120F5E7878947F0D4
:106A2000100787810220EFE7042727700C4C2570A0
:106A3000C48844F40064C480886840F0040088601E
:106A4000C8E70000102C01402C0700204007002060
:106A50003F070020000C0020A4020020C80A0020EC
:106A60005D070020704700002DE9F0434FF08040A3
:106A7000018A21F001010182AA48007800287CD116
:106A8000A94FF87B002878D1A848406C322874DCE4
:106A9000A7488068DFF89C924104A74DB9F804002C
:106AA0004FF0000403D4401CA9F8040024E100289E
:106AB00074D02978012611B1012912D013E1494679
:106AC000B0F5BE7FFAD92E70CC718C71EC702C723F
:106AD000287A0A18401CC0B2147228720F28F7D303
:106AE00001E1B9F802204946824201D9EE7100E085
:106AF000EC7190488A7908300F2A15D2CB79082B8F
:106B00000BD2C3F10708EB7912F800C003FA08F3BF
:106B100063441354CA79521CCA71CA79082A03D132
:106B20008A79521C8A71CC7199F80610C8460F29CF
:106B300073D10D21FBF71AFAA881010A6970C0B25E
:106B4000A87088F8064098F816208A4265D198F80F
:106B50001510814261D198F80BC0784903230222B5
:106B60007748BCF1000F10D0BCF1010F02D0BCF18E
:106B7000020F14D080F86A2000E0C7E091F800C04E
:106B80002CF00C0C0CF1080C0FE080F86A6091F806
:106B900000C02CF00C0C0CF1040C06E0A5E080F811
:106BA0006A3091F800C04CF00C0C81F800C098F8E5
:106BB0000C10B6EB111F04D180F86E4087F84A40E4
:106BC0000EE0B2EB111F04D180F86E6087F84A60C6
:106BD00006E0B3EB111F03D180F86E2087F84A203E
:106BE0000B0717D001F00F01012901D0022915D0A0
:106BF00080F86C602C7198F80D102A7906FA02F36F
:106C00000B406B71082A41D2DFE802F00B0F4016EF
:106C1000212C333A80F86C40ECE764E080F86C207B
:106C2000E8E713B380F8704030E013B180F85060AB
:106C30002CE080F8504029E023B180F8656087F8A7
:106C4000076123E080F8654087F807411EE023B123
:106C500087F8F94080F84D4018E087F8F96080F82F
:106C60004D6013E013B180F868600FE080F8684071
:106C70000CE013B180F8666008E080F8664005E03B
:106C800013B180F8676001E080F86740521CD2B20F
:106C90002A71082AB1D398F80E108A0704D587F80C
:106CA000F56080F8646005E0264A87F8F54080F8D2
:106CB00064405481C90702D080F8294001E080F87F
:106CC000296098F8111000F86D1FC2781E48012A3B
:106CD0001ED001B3012921D04FF48051A0F87610C5
:106CE0001A493C200870A9F80240A9F80440B9F8F4
:106CF0000210491CA9F80210B9F80210B1F5FA7F88
:106D000004D940F2F511A9F802102C70BDE8F08307
:106D100044F21C71E2E74FF40051DFE741F25551B4
:106D2000DCE700003F070020A4020020380100201B
:106D300000100140400E0020C8060020D0040020B2
:106D4000580E0020000C0020380500203C070020D1
:106D50002DE9F05FFCF704FD8E4D2888A5F10406AF
:106D6000C0070AD0308820F008003080288820F042
:106D70000900288002F0BAF8D9E02888DFF81892D4
:106D8000DFF81882864C80071AD5B9F8001041F058
:106D90000101A9F80010B8F8000080491431503002
:106DA000088028884FF6F95108402880308840F044
:106DB00004003080FEF726FF84F83C00BDE8F09F19
:106DC0002888784F4007288871D520F00400288053
:106DD000FEF718FF94F83C108142EFD1308820F084
:106DE00004003080FCF7DCFE2078410605D594F8DD
:106DF000541094F83B209142E0D03978400621F0BD
:106E00000201397004D5FDF749FE97F82F7004E0B0
:106E100094F83C00FCF7F6FC0746DFF880B140F63A
:106E20008C2A0BF1180B062F47D294F83800B84281
:106E30003ED03846FCF76AFC2078C00716D094F89C
:106E40003A0094F8391000F00302914206D0A17A7A
:106E500000F0010001F00101884215D1FCF708FEA5
:106E6000F9F7E8FFFCF730FF384689E0FCF700FE51
:106E7000F9F7E0FFFCF728FF3846FCF719FE207809
:106E800040F00100207099E7288820F00800288051
:106E9000206B810801EBD000504515D2B8F80010E6
:106EA0000844ABF80000308840F0080003E00DE033
:106EB000308820F00800308080E7B9F8001041F0F9
:106EC0000101A9F80010DFE75046E7E7000728882E
:106ED00031D520F008002880308820F0080030806C
:106EE000FEF790FE84F83C00FCF75AFE387820F05C
:106EF000020038702078400604D5FDF7CFFD97F8E2
:106F00002F5004E094F83C00FCF77CFC0546062D6D
:106F100008D294F83800A842B5D0FCF7A9FDF9F7DB
:106F200089FF2AE02048C18841F04001C180BDE8C6
:106F3000F05FFCF7A9BEC006288825D520F0100018
:106F40002880308820F01000308097F838000C2816
:106F500002D2401C87F83800387840F002003870C0
:106F6000FDF79CFD97F82F50787884F8390094F855
:106F70003800A84287D0FCF77BFDFCF7A5FE284629
:106F8000BDE8F05FFCF794BD4EF2BE1108402880CA
:106F900014E70000100400400004004024040040F6
:106FA0003801002058040020000C00202DE9F04F8B
:106FB000514F85B0388820F0010038804E480026B7
:106FC000103006804D4CDFF838A14FF0010894F8DE
:106FD0005C0042F63029C10774D072B64948816915
:106FE00041F400718161816941F4806181614FF4F4
:106FF0000040FEF7C1FD444D00212846F9F766FC2C
:1070000000212846F9F758FCDFF800B10021584666
:10701000F9F752FC00213E48FBF772FC2846F9F7CD
:1070200077FD5846F9F774FD4FF46020CDE902066C
:107030008DF8056000968DF810808DF80480694603
:107040002846F9F7F7FD01231A460F212846F9F7DC
:1070500042FE01212846F9F72FFC00204946401C3A
:1070600080B28842FBD328462E600121F9F772FED8
:1070700028688007FCD524484C30006894F85C10E0
:1070800021F001012144A1F85000F9F729FC62B672
:10709000FDF710FC47F69061AAF8001094F85C0028
:1070A000401CC0B284F85C000C2822D21249143172
:1070B000A1F80080388840F00100388005B0BDE8B4
:1070C000F08FFFE7134920F00100085A12490880A9
:1070D000114945F65800083908800F4846F658010E
:1070E000001F01800C4920200C390880AAF800906C
:1070F000D4E70320A070E1E7000800405804002016
:107100002C080040001002400024014000280140EB
:1071100008000240BCAF0008202C01400029018873
:1071200002D041F0800101E021F080010180704730
:1071300010B50A884B88CC881A438B8823431A439E
:107140000B891A434B8989891A430A43A0F84420C2
:1071500010BD0021018041808180C1800181418179
:10716000818170470029818802D041F0010101E04E
:1071700021F00101818070470029018802D041F08F
:10718000010101E021F0010101807047002930F880
:10719000441F02D041F4004101E0C1F30E0101801F
:1071A000704700004B4910B5884202D10121C41438
:1071B00086E0B0F1804F09D0474988420DD10121C6
:1071C0000220FEF7FBFC0021022064E001210846BA
:1071D000FEF7F4FC002101205DE04049884206D121
:1071E00001210420FEF7EAFC0021042053E03C4981
:1071F000884206D101210820FEF7E0FC002108208A
:1072000049E03849884206D101211020FEF7D6FC1A
:10721000002110203FE03449884206D1012120207E
:10722000FEF7CCFC0021202035E03049884202D115
:107230000121441444E02E49884202D10121CC04AA
:107240003EE02C49884202D101210C0538E02A4950
:10725000884202D101214C0532E02849884206D1FA
:1072600001214020FEF7AAFC0021402013E0244920
:10727000884206D101218020FEF7A0FC0021802059
:1072800009E0204988420AD1841501212046FEF7F1
:1072900095FC00212046BDE81040FEF78FBC1A493E
:1072A000884202D101210C040AE01849884202D127
:1072B00001214C0404E0164988420AD101218C04C2
:1072C0002046FEF793FC2046BDE810400021FEF763
:1072D0008DBC10BD002C014000040040000800409F
:1072E000000C004000100040001400400034014039
:1072F000004C014000500140005401400018004083
:10730000001C0040002000400040014000440140BB
:1073100000480140002A828901D00A4300E08A43E4
:107320008281704730B5028C22F001020284028C07
:107330008388048B22F0020224F073050C882C430E
:107340000D8915434A882A43114DA8420BD0114D8F
:10735000A84208D0104DA84205D0104DA84202D036
:107360000F4DA8420DD122F008054A8923F440733D
:107370002A4322F004058A882A438D891D43CB893C
:107380002B4383800483C9888186028430BD00003A
:10739000002C014000340140004001400044014005
:1073A00000480140028B22F008020A430283704722
:1073B00070B5028C22F010020284028C8488038B48
:1073C0000D8823F4E6464FF6FF7303EA052535439F
:1073D0000E8922F0200203EA061616434A8803EAC1
:1073E00002123243104EB04202D0104EB04215D1BC
:1073F00022F080064A8924F4406403EA02123243F0
:1074000022F040068A8803EA021232438E8903EA98
:1074100086062643CC8903EA8404344384800583AA
:10742000C9880187028470BD002C014000340140EE
:10743000028B4FF6FF7322F4006203EA012111432D
:107440000183704770B5028C22F480720284028C32
:107450008488838B0D8823F073031D4322F400730B
:107460000E894FF6FF7202EA06261E434B8802EA97
:1074700003233343104EB04202D0104EB04215D118
:1074800023F400664B8924F4405402EA0323334377
:1074900023F480668B8802EA032333438E8902EA51
:1074A00006162643CC8902EA04143443848085837B
:1074B000C9888187038470BD002C014000340140DD
:1074C000828B22F008020A438283704770B5028CD7
:1074D00022F480520284048C8288838B0D8823F4EA
:1074E000E6464FF6FF7303EA0525354324F40056BC
:1074F0000C8903EA043434434E8803EA06362643F3
:10750000094CA04202D0094CA04205D122F480448B
:107510008A8903EA8212224382808583C988A0F87F
:107520004010068470BD0000002C01400034014072
:10753000828B4FF6FF7322F4006203EA01211143AC
:1075400081837047018582827047828822F07002B1
:10755000828082880A4382807047A0F8401070477A
:1075600030B502881B4B1C4C98420DD0A0420BD06A
:10757000B0F1804F08D0194DA84205D0184DA8424F
:1075800002D0184DA84203D122F070054A882A4340
:10759000154DA84206D0154DA84203D022F44075DF
:1075A000CA882A4302808A8882850A88028598428E
:1075B0000AD0A04208D00E4A904205D00D4A90420F
:1075C00002D00D4A904201D1097A018601218182BF
:1075D00030BD0000002C0140003401400004004098
:1075E00000080040000C0040001000400014004063
:1075F0000040014000440140004801404FF6FF7147
:10760000818000210180C180418001727047002982
:10761000018802D041F0020101E021F00201018065
:1076200070470029018802D041F0040101E021F0F7
:1076300004010180704780092830FF2801D9FF200C
:107640007047C0B270472DE9F041B1F902500023F4
:107650001E240F22854203DDB1F90000BDE8F08150
:10766000B1F97A50854202DAB1F97800F6E701EB18
:107670008205B5F90250854201DA134600E014464E
:10768000E21852085D1CAA42F1D101EB8203B3F962
:107690000240844206DAB3F9067031F92250B3F998
:1076A000046005E033F9027C31F9225033F9046CAF
:1076B000001BC11789013A1B41EA9061D317800171
:1076C000F8F730FD721BA0FB024601FB0261D317E5
:1076D00000FB0310810641EA9410284400B2BDE784
:1076E0002DE9F04FDFF8B8B16A48DFF8AC91DFF868
:1076F000ACA190F80EC0BBF91A70BBF91C60BBF9C5
:107700001850BBF96C10BCF1070F48D2DFE80CF041
:107710008D041A30485E7600D9F80020C284DAF869
:1077200000200285C28C038DA7EB820212B2A6EB69
:1077300083034A431BB2594342F3CF2241F3CF2381
:10774000D11870E0D9F800208284DAF80020028590
:10775000828CA5EB820213B2028D4B43A6EB820210
:1077600012B243F3CF24514341F3CF23E11814E085
:10777000D9F800200285DAF800208284028D838CFB
:10778000A6EB820212B2A5EB83031CB24A4361430B
:1077900042F3CF2341F3CF24191949420AB244E0FE
:1077A000D9F80020C284DAF800208284C28C838C4D
:1077B000A7EB820212B2A5EB83034A431BB25943E3
:1077C00042F3CF2241F3CF24111914E0D9F800205D
:1077D0008284DAF80020C284828CC38CA5EB8202FA
:1077E00012B2A7EB83034A431BB242F3CF2459439F
:1077F00041F3CF22A11849420BB216E0D9F800207C
:107800000285DAF80020C284028DC38CA6EB8202C6
:1078100012B2A7EB83031CB24A4342F3CF23614366
:1078200041F3CF22991849420CB2BBF91E50594678
:1078300005F21E56A64201DACE8306E0A5F21E55D9
:10784000A54201DDCD8300E0CC83B1F9204004F2F4
:107850001E55954201DA0D8406E0A4F21E549442AE
:1078600001DD0C8400E00A84B1F9222002F21E54EA
:107870009C4202DAABF8224008E0A2F21E529A4281
:1078800002DDABF8222001E0ABF82230417B8173AE
:10789000BDE8F08FA40200203C2401403C280140B8
:1078A000380500202DE9F04704467048714E002746
:1078B00002786F48022AB0F9341004D0082A6ED03A
:1078C000092A6DD0CDE0C27B022A02D1B0F8442053
:1078D0005AB1A4F8421071810423B6F908101A466F
:1078E0000020FEF71DFF3081BBE06349DFF88C818B
:1078F000496A0D14E58090F84A1099B10089DFF8C3
:107900008091C0F3C001C0F30020814223D1D8F898
:10791000440040F2BA41884240DD40F66A11884294
:107920000ADC15E0B4F9020040F2DA21884279DD80
:1079300040F26A41884204DD0823B4F942101A4635
:107940004EE0A0F2DA20F8F776FD00224D4B56E02B
:10795000A0F2BA404FE04C480078C0060CD5D8F8E9
:10796000440041F2243188425CDD41F2D471884206
:10797000E2DC00F6DC4020E04448DFF8149190F8A7
:10798000701001290DD090F86F00012809D04148EE
:107990000178C90746D04049098889B142E05AE0D8
:1079A0005DE0B4F9020041F6DC6188423ADD42F262
:1079B0003411884210DC00F59270A0F500501AE0F6
:1079C000B0F91000B4F90210A0F59672914229DDC9
:1079D00000F5967291420BDDB4F9421020231A464D
:1079E0000020FEF79DFEA4F84200002817DB1BE0F4
:1079F000081A00F59670F8F71EFD00224B46F8F7BE
:107A000086FC0E22F8F7F2FCF8F74CFD00B2C0F548
:107A1000804068438013A4F84200002D04DCA4F8E1
:107A2000427001E0A4F842501C48B0F91210D8F896
:107A30005000081A718B01EB600000B2F082002840
:107A400000DCF782B4F94200B6F91610884200DB78
:107A50000846708104E01248B0F87C00F9E77181B3
:107A6000378184F84070BDE8F08700003F070020B0
:107A7000A40200204C00002038050020380100201E
:107A800000C092400000794010070020580E0020EE
:107A900000C08240B00A002008000020C80A002070
:107AA000140C00202DE9F041B1F9025000232B24E1
:107AB0001522854203DAB1F90000BDE8F081B1F981
:107AC000AE50854202DDB1F9AC00F6E701EB82056C
:107AD000B5F90250854201DD134600E01446E21874
:107AE00052085D1CAA42F1D101EB8205B5F90230C2
:107AF000834206DA35F9026C35F9044C31F922106B
:107B000006E01E4631F92240B5F90630B5F90410F9
:107B1000801B091BC5178911AD0345EA90458703F2
:107B2000A1FB070CCA1702FB07C201FB05219A1B28
:107B3000D317F8F7F7FA000A40EA0160001900B21B
:107B4000B0F5804FB9DB43F6FF70B6E770B5134C64
:107B500040F224452946204600F02CF800281BD08E
:107B6000204600F046F82946204600F01DF80C4C4F
:107B700000212046FAF7C4FE2046FAF73FFFC0F185
:107B800064000849C0B20428087201D900F0AEF9B7
:107B9000BDE87040FAF770BF70BD000000380140CA
:107BA00058000240740600200A0A01219140C9438E
:107BB0000180704730B501F01F0201240025C1F398
:107BC000421304FA02F2012B0FD0022B0FD0838A4A
:107BD0004FEA11210088134204FA01F400EA04007C
:107BE00001D000B10125284630BD8389F0E7038A22
:107BF000EEE78088C0F308007047000070B5214CA4
:107C00002068214D400103D520492846F9F75CFA48
:107C10002068000104D51D492846FF31F9F754FAC0
:107C20002068C00003D51A492846F9F74DFA1948CB
:107C3000194A0178CB0712D192F82F30012B0ED0C0
:107C4000FAF762F92068C0F382611448072916D058
:107C5000216811F0E05F01D15521017070BD012351
:107C600082F82F3021F0010101700D4801680D4AA2
:107C700001F4E06111430160BFF34F8FFEE7002183
:107C8000EBE7000008640040006400400100003899
:107C9000000001383E080020CC0E002048080020DB
:107CA0000CED00E00400FA05F0B585B004200025D5
:107CB0008DF808000702844C009501958DF80A5054
:107CC0008DF8135039462046F9F75EFB01281DD187
:107CD0007E4E06F8305FF9F775F9206840F40040F1
:107CE000206079481430016821F001010160784D6D
:107CF000286800F0FBFD002176A001F051FE28600D
:107D000039462046F9F7F8F9012030700221204663
:107D1000F9F73AFB01287CD16A4600212046F9F7A1
:107D200009FC01986E4920F0604088609DF80A10B7
:107D300008291BD16B4908440C2817D2DFE800F052
:107D4000060BBDBDBDBDBD1752717CA364489DF837
:107D50000B106F309BE0624A0020694617320B1807
:107D6000DB7A1354401CC0B20828F8D3A5E05C4964
:107D70009DF80B004F3103090A7860F3030263F3A7
:107D80000412430963F34512800960F387120A70F5
:107D90009DF80C0048709DF80D0088709DF80E004D
:107DA000C8709DF80F000A7960F30002400860F384
:107DB00047020A719DF8100048719DF811208879DA
:107DC000930862F3010063F38300120962F3071062
:107DD00088719DF81220C87962F30600D20962F317
:107DE000C7104EE040489DF80B1001709DF80C1034
:107DF00041709DF80D1001F003028270C1709DF872
:107E00000E1001719DF80F1041719DF810108171D5
:107E100000E056E09DF81110C1719DF8121001723A
:107E20004BE02F489DF80B205730017862F3010199
:107E3000920862F387012AE029499DF80B205F31FF
:107E4000087862F30300120962F3071008709DF8C6
:107E50000C0048709DF80D20887862F30600D20966
:107E600062F3C71088709DF80E00C8709DF80F006F
:107E700008719DF8100048719DF8110088719DF8F7
:107E80001200C87119E016489DF80B106730017098
:107E90009DF80C1041709DF80D1081709DF80E102A
:107EA000C1709DF80F1001719DF8101041719DF87F
:107EB000111081719DF81210C17102212046F9F74D
:107EC0001BF905B0F0BD000000640040CC0E00209E
:107ED0004C0800206465765F63616E31000000002D
:107EE00060070020FFFE00E71010002070B51D4D58
:107EF00000242878432834D16878462831D1A878DE
:107F0000502807D0512805D0812803D0892801D0D6
:107F1000212826D1144E7071E9787172A81C891C31
:107F2000FAF75CF8B072717A294409793182884293
:107F300017D106F10E00017841F0020101700B48E3
:107F4000016841F020010160317A0948002204E013
:107F50002B5D03552A55641CE4B28C42F8D380781B
:107F6000707170BDF0080020740600200C0C0140F8
:107F7000920D002070B51D20FDF7D0FAFCF78EFDA4
:107F80001D20FDF7E1FA154890F82F10144D062337
:107F9000144C85F8381090F83B1095F83B201143AD
:107FA000012A04D0022A07D0042A0AD010E0827ADB
:107FB0008A420DD0007B09E0027D8A4208D0807D94
:107FC00004E0827F8A4203D090F82000884200D1EA
:107FD0002370002085F8400070BD00005804002088
:107FE000380100203F0700200B4800214180A0F10C
:107FF000B8018A898280CB891A44C2800B8A1A44CC
:1080000002814B8A1A444281898A1144818143F654
:10801000FF71C18170470000F0010020084940F65F
:108020001C72B1F90C00904202DA00F59F7005E075
:1080300041F2E302904201DDA0F59F70C8817047D4
:108040004C00002038B51348C16941F00401C161FA
:108050001E208DF8000002208DF801008DF802002E
:1080600001248DF803406846FDF77AFA0A49842016
:108070000880094947F690602C3108800020091FCC
:108080000880054914310C80091F0880081F0480EE
:1080900038BD0000001002400008004030B4204904
:1080A0001E4A45788B7A114692F83B4091F8391078
:1080B000AC4218D14BB10379994202D0437999422D
:1080C00001D140791AE0807909E08379994202D0A0
:1080D000C479A14202D182F82F3011E0407982F8B0
:1080E0002F0030BC7047C578AC42FAD16BB1C37970
:1080F000994202D0037A994205D1007A82F82F0082
:1081000030BCFEF7BFBB407AE9E7437A9942E2D040
:108110000479A142DFD0007AE1E700005804002092
:1081200038010020FEE700002DE9F0470446007FFB
:10813000012868D13548E1880288511A89B2072997
:1081400016D30088E080B4F9000044F2DD414843D2
:10815000401346F6D96148438013A060401000B236
:10816000A0814FF08051B1FBF0F0F8F75FF920618A
:10817000B4F90C6096B1B4F902104DF6B050484312
:108180000014A082B4F904704DF6B05207FB02F25D
:108190004FEA2245E58204D4024603E00020E08352
:1081A00030E0424212B22283002D01DB2B4600E078
:1081B0006B421BB2DFF85890638398464FF4804AB5
:1081C000B24208DAF8F729F92169F7F7FCFFF8F766
:1081D00050F9801304E0002901DA484600E05046D7
:1081E000E083B04509DA2846F8F717F92169F7F76F
:1081F000EAFFF8F73EF9801304E0002F01DA484661
:1082000000E050462084BDE8F087000048070020C9
:1082100000C0FFFF2DE9F0414C484D4E002500788D
:10822000A6F15004022806D14A4FF87B022802D159
:10823000B7F8440030B1A5862564B56284F838509B
:10824000BDE8F08144488168C068494300FB0010E4
:10825000FBF75EF940F233314843810BB4F8440038
:1082600043F6CC42504301EB903080B243F6991173
:10827000A4F84400884209D338481146B0F90400F4
:10828000884203DB97F84A00032813D00123B4F98E
:1082900034101A460020FEF743FAA086B4F84000D6
:1082A000012301B21A460020FEF73AFA2064800347
:1082B000B06226E0B4F8460041F69A13A0F51852D1
:1082C000663A9A4209D2B4F94400214AFAF7C0FF4B
:1082D0002064012084F8380022E044F247118842EB
:1082E00012D994F83800D8B11D480178491CC9B298
:1082F0000170022914D30570206C10B1401E206457
:1083000008E084F838500BE0A0F58040B0F5A47F79
:1083100003D2206C8003B06202E084F83850B5626A
:10832000B4F840000A4980B20839323401F006FD41
:10833000B4F90000B4F91810414389136180B4F90D
:10834000161048438013A0807AE700003F07002002
:10835000800A0020A4020020BC090020E2050020C1
:10836000320100200D480021A32280F82810C1838B
:1083700081865030C2600E22028241F26202426166
:1083800008220283418341F2555282839203C0E95D
:10839000081240F28E32826081627047300A0020FB
:1083A0002DE9F0410546FBF7ABF9204C204E07467E
:1083B00020686168421C8A4220D009B93F281DD03C
:1083C00004EB0010AA7A05F10B010E30F7F7DBFE83
:1083D0002168686804EB011188602168A87A04EBC1
:1083E0000111888172B62068401C2060402801D3AA
:1083F0000020206062B6307888B114E03846FBF780
:1084000067F90A28D4D3706800F070FA002109A037
:1084100001F0C6FA70604FF0FF30BDE8F0815520E2
:108420003070F9F771FD0020F7E70000A814002074
:10843000480800206465765F63616E3100000000CB
:1084400010B504000B462D4AC3F1000028D5644244
:10845000002B12DAA04207DA214600F0F1FB32F8D5
:108460001000C0F5404041E00146204600F0E8FB26
:1084700032F8100000F5004038E0A34208DA214647
:10848000184600F0DDFB32F8100000F540402DE00A
:10849000204600F0D5FB32F81000C0F5803025E012
:1084A000002B12DAA04207DA214600F0C9FB32F8AD
:1084B000100000F5804019E00146204600F0C0FBA6
:1084C00032F81000C0F5004010E0A34208DA21465F
:1084D000184600F0B5FB32F81000C0F5804005E00A
:1084E00053B1204600F0ACFB32F81000B0F5004F5D
:1084F00001DDA0F5803010BD002010BDC8AF000820
:1085000040438013494300EBA13000220302002BBB
:1085100014DDB3F5001F01DC802001E04FF40050B2
:1085200093FBF0F1014401EBD1714910814206D077
:10853000521CD2B20846062AF2D300E00021C8003D
:1085400000B2704702E008C8121F08C1002AFAD121
:1085500070477047002001E001C1121F002AFBD1C3
:10856000704700002DE9F047BD4CBE4821880288C5
:10857000511A89B20F297DD30088A4F13C052080CF
:10858000288F08B1401E28872B78B74AC3F3810093
:1085900001281ED0022821D0118BB148B44EDFF83B
:1085A000CC92407EB6F806C00027B1F5926F1CD879
:1085B000142818D3782060764CF01000F08040F238
:1085C0006660A88123F001002870D77389F80070D5
:1085D00018E0108B00EB4000C00302E0108BA549AF
:1085E0004843010CD9E7401C04E0B1F5216F09D9DB
:1085F00010B1401E607605E02CF01000F08043F0D2
:1086000001002870B5F90200B5F914304143C3EBFD
:10861000C303C1F38F31C3F3D10303EB510109B29B
:10862000A9829046128B4FF080535043B5F9162023
:10863000C0F38F30C2EBC202C2F3D10202EB500092
:1086400000B2E882AA6A42431213EA6293FBF2F292
:108650002A63894A1080A2680A44A260E168014442
:10866000E160207C401CC0B22074072802D942F38C
:10867000CF0000E0E8E02883C9106983E760A760C5
:1086800041F6C8012774884204DD2A8B7B49B1FB7F
:10869000F2F1E981C117890341EA9041800342F672
:1086A0009B420023F7F73EFDA8846D482A78A0F18D
:1086B0003C009307B0F90600C2F3810200EB801181
:1086C00001EB003141F30F3115D5012A07D0022A01
:1086D0000BD04EF6AC3141430914A18011E049F2B0
:1086E000586250430014A08020E04CF20C3141430A
:1086F0000914A18026E0012A0ED0022A18D0A080F9
:1087000069845F4948430014A4F81E00FAF736FB59
:108710005C480088C0B143E04AF2904242431214E0
:10872000A2804BF2C822504300146884E183EDE735
:108730004CF6345141430914A1804DF66C3141434C
:10874000091469845049DDE795F8200000BB88F8DA
:108750000F7089F80070B5F91A00A0F514512C3982
:10876000B1F56E7F18D2617FF42912D94749E880AC
:10877000434AA1F8460050430014A880A1F84400E1
:10878000FF2085F8200081F8280041493C2008702E
:1087900006E0491C617703E0607F08B1401E607706
:1087A000B5F91A00B4F91E203A4990420DDDA27EB7
:1087B0007D2A08D9F28842F00802F2800A7822F075
:1087C00002020A700EE0521C06E0A2F23D12904234
:1087D00008DAA27E12B1521EA27603E0F28822F0DD
:1087E0000802F280B4F90420904214DA2A4B9B6804
:1087F000B3F5FA7F0FDAE07E3E2809D9F08840F021
:108800001000F0802777087820F0020008700CE054
:10881000401CE07609E002F23D12904201DD8888BA
:10882000A0B1207F08B1401E2077B5F9181060690B
:1088300008446061217E491CC9B221761F2903D9F1
:108840004011A88367612776BDE8F087207F7D28E7
:1088500004D9F08820F01000F080E6E7401CE3E740
:108860000C05002048070020A40200203F0700203C
:10887000000C002030330100700B002074E8260B40
:10888000188601004A070020E0380100580E002039
:108890003C070020E205002038050020024941F293
:1088A000F460886270470000D004002070B50D4C61
:1088B000207828B1012808D0062505280FD10BE023
:1088C0000948F9F79BFD012004E00748801DF9F7EE
:1088D00095FD0520207070BDF9F7B0FD257025705D
:1088E00070BD000040070020D0AE00080A4A4FF0DB
:1088F000FF31B0EBA20F0CDA00280ADB0749096848
:1089000051F820004068006900B100476FF0050091
:108910007047084670470000040000007C080020F3
:1089200070B50A4DA86870B100240948AC60F8F72A
:1089300073FC084804604460A0F5816004604460F2
:108940002C70002070BD6FF0040070BD480800203E
:1089500000640040A81400207FB505460024631E73
:10896000244A4FF00050072D41D2DFE805F04004C3
:10897000111E21403C00814208D2D068202805DA2F
:108980001D4B43F82010401CD0600CE01C4627E033
:108990008142FBD210692028F8DA174B803343F864
:1089A0002010401C10610023F0E7F8F74BFC17E0A3
:1089B00000208DF80B000121ADF800000422ADF875
:1089C0000400ADF808008DF80C108DF80A00ADF821
:1089D0000220ADF806208DF80D106846F8F76EFC01
:1089E000204604B070BDBDE87F40FAF71DBF1846B1
:1089F000F7E7000048080020B0180020F8B5414E05
:108A0000B06801287BD04048F8F706FC0121082017
:108A1000FDF7E0F801210846FDF7DCF801214806E2
:108A2000FDF7C0F801214FF4EA10FAF715FE4FF4F4
:108A30008070ADF8000003248DF802400420334D0F
:108A40008DF8030069462846FAF7B4FD6815ADF8BD
:108A500000008DF8024018208DF803006946284672
:108A6000FAF7A8FD14208DF8000002278DF8017098
:108A700000248DF8024001258DF803506846FCF76C
:108A80006FFD13208DF800008DF801708DF80250F5
:108A90008DF803506846FCF763FD16208DF8000042
:108AA0008DF801408DF802408DF803506846FCF7C0
:108AB00057FD17490120FFF74FFF16490120FFF727
:108AC0004BFF15490120FFF747FF14490120FFF72D
:108AD00043FF13490120FFF73FFF00210320FFF769
:108AE0003BFFF8F745FB0F4804604460A0F5816048
:108AF0000460446034700020B560F8BDFFE74FF0BB
:108B0000FF30FAE74808002000640040000C0140F4
:108B100020FF401820FF431820FF441820FF45186D
:108B200020FF2518A81400202DE9F04781461E4893
:108B300086B0174680680E46A0B14FF0FF381FB3CD
:108B40006846FAF77FFE401C0ED00DF10B019DF830
:108B50000A208A464846019DF7F715FB9DF80A4012
:108B60003D601DE06FF0040006B0BDE8F08700BF77
:108B7000FAF75AFE411C15D0A84213D16846FAF7FD
:108B800061FE0198A84201D04046EDE79DF80A2019
:108B900009EB04005146F7F7F6FA9DF80A00044481
:108BA000B442E5D32046DFE7480800202DE9F0472E
:108BB0000646224886B00024806888B1601E002ADC
:108BC00010D012680192B2F1005F0BD2CF0801F011
:108BD00007054FF000084FF004094FF0080A17E0AE
:108BE0006FF0040006B0BDE8F08700BF8DF80AA062
:108BF0008DF8089006EBC4008DF809800168CDF867
:108C00000B104068CDF80F006846FFF7C9FB641CE5
:108C1000BC42EBDB7DB18DF80A508DF808908DF8E1
:108C2000098006EBC4012A460DF10B00F7F7ABFAF9
:108C30006846FFF7B5FB0020D4E700004808002095
:108C4000090A05D0B0FBF1F0FF2800D9FF207047DA
:108C500000207047D0E90021C368521A5A4301EB43
:108C6000A231816041607047B0F90020B0F9021074
:108C7000B0F90630521A5A4301EBA231818041808B
:108C80007047000030B5494B188849498A89801AD5
:108C900085B24848484A0F2D047801F14C001DD395
:108CA0001D888D81117A090713D5022C01D0434903
:108CB00012E0434DB0F90210B5F90050A94205DCAD
:108CC00002DA01F1020108E0458007E0A1F10201AA
:108CD00003E0022C02D13B4909884180B0F84010E2
:108CE0001D88691A89B29C2949D31988A0F84010B7
:108CF000D16A0023B1F5804F31DB3349096DB1F5FD
:108D0000405F2CDD314940F26665B1F91010A9428F
:108D100012DD43F69915A94202DB40F2333108E037
:108D200040F23335A1F26661694343F2333591FB7A
:108D3000F5F1A0F8441001E0A0F844302449B2F85D
:108D40000A510978C1F381012DB100BFB0F8441078
:108D500001F21E511CE092F84A20032A10D0A0F81C
:108D60004430022C01D0A0F84430B0F95C10B0F9C6
:108D7000443001F114029A420DDAA0F85C2030BDB3
:108D8000012901D00229E1D1B0F8441001F23331B8
:108D9000A0F84410E5E703F11402914203DD143911
:108DA000A0F85C1030BDA0F85C3030BD4807002052
:108DB000000000203F070020A4020020CE04002075
:108DC000CC040020C8040020380100203805002011
:108DD000D00400202DE9FC4101210220FCF7E2FE35
:108DE00001211920FCF7F6FE01213C48FAF734FC7A
:108DF0004027ADF8007003248DF802400420384D60
:108E00008DF8030069462846FAF7D4FBE001ADF877
:108E100000008DF802401C208DF8030069462846AA
:108E2000FAF7C8FB4FF4E0712846FAF74AFCA81598
:108E3000ADF800008DF8024010208DF8030069465F
:108E40002848FAF7B7FB4FF4A060FCF7BBFB1D20E6
:108E50008DF8040001268DF8056000258DF8065078
:108E60008DF8076001A8FCF77BFB1F498C20088068
:108E70001D494FF6FA702C3108806E20091F0880BA
:108E800019481430068018480830078016492031E8
:108E90000D80154AD020121D1080134A45F2F300B0
:108EA000183210800A1F45F2500010800E4A4FF60B
:108EB000FF7038321080121D1080121D108041F298
:108EC0001B10088000F012F8FAF7DEFE064810309A
:108ED0000580001F0480BDE8FC810000000C1A0022
:108EE00000100140000C01400004004070B51D203E
:108EF000FCF709FB2A4D40212846FAF7D9FB8400EC
:108F000080212846FAF7D4FB44EA4004A9152846F4
:108F1000FAF7CEFB0443E0B2224C84F83C00FAF7A7
:108F200071FC0546052805D91F48C18841F040015C
:108F3000C18001E084F838501C48007A000703D54E
:108F400094F838001A490D5C4FF6FA702063E0621D
:108F5000A06260622062E061A06116486063002048
:108F60006064206584F83F0084F84000FAF7F8FB5D
:108F7000A07AFF2811D0022084F83D000E48008816
:108F8000A0662846FBF7E2F8207820F00100207068
:108F9000BDE870401D20FCF7CCBA0120ECE70000D2
:108FA0000010014038010020000C0020A402002025
:108FB000C4B80008DCFF0500240400402DE9F0439C
:108FC0004D484E4902880B889A1A92B20F2A67D3ED
:108FD000098801804A49C98B027D00EB42029180D9
:108FE000017D491CC9B20175082959D300240475B3
:108FF0002246017D00EB4103491CB3F90430C9B29C
:1090000002EB630212B201750829F2D33D490475DF
:109010003D4B4A8044800E789D895FEAC67C40F6CD
:1090200038694FF0030714D0A2F22B5C42F6E858DF
:10903000C44520D3A1F1020C26F00204ACF80020B4
:1090400047750C7040F22B54A24211DA45F004022D
:109050001EE046F001060E704A4507DD45F00102AC
:109060009A8126F002020A70477517E0447515E0F0
:1090700045F002020CE04A450CDA8775427D12B1D8
:10908000521E42750AE046F002020A7025F00702FD
:109090009A8103E0837D2BB15B1E837540888880B5
:1090A000BDE8F08342F6AA239A4222DAB1F90430ED
:1090B0002BB941F2CD05AA4201DA4480EEE7134C08
:1090C000920302EB843241F67244B2FBF4F214B222
:1090D0004FF4805502464480AC4200DA5580B2F924
:1090E0000240E41A04F5A374B4F5237FD6D8438074
:1090F000D4E74FF48043FAE7940C0020480700209F
:10910000A4020020E2050020000C0020C8F1FFFFAF
:109110002DE9F0416D4CDFF8B8E14FF0000594F80F
:109120003410C80706D094F938104B42002958DD96
:109130000E4657E0674884F83750A4F84250664A14
:1091400090F8380084F840009586CEF80450CEF8A8
:109150000850624E40F26663CEF80C50A4F87C30A2
:1091600036F810005E4E768830444FF6FF7606EAF9
:10917000800024F8300B4FF0806044F8040CA320EA
:10918000208460845810A084E38440F699102085E0
:10919000580060854FF48050A08541F23330E0855F
:1091A00041F26660208641F69910608641F6CC4017
:1091B000A0864FF40050E08642F23330208742F21E
:1091C0006660608742F69910A08742F6CC40E0873F
:1091D00082F8A15041F00100207184F84450BDE8AC
:1091E000F0811E4694F937004242002801DD07460F
:1091F00000E01746F61B012E0BD0002800DB0246CC
:109200005FFA82F684F8380094F84F00012805D000
:1092100041E0002900DA1946CEB2F3E794F939307B
:109220005942002B01DB184600E0084694F93A2029
:10923000C7B25042002A01DB944600E08446BC4598
:1092400008DD002A00DA0246D7B2002B00DA0B460E
:10925000D8B207E0002B00DA0B46DFB2002A00DBB1
:109260001046C0B204EB4000B0F9501004EB4700C8
:1092700030F9502F11444910018084F84F5084F880
:109280003E5084F83D5084F83C5084F83B5084F8BC
:109290003A5084F8395004EB46007546B0F9500056
:1092A00024F8420FBEF80410C82309B26422FDF767
:1092B00037FA6860E968401AA9680844A860B5F9F7
:1092C00000104843C013E860608788E7140C002052
:1092D000D005002038010020A4020020D6B80008E4
:1092E0004C000020F0B4544890F83410C90776D0F0
:1092F000524990F84030002291F838108B426FD0DC
:109300004F4CA0F872204F4DE65C04468E4294F913
:10931000374002D0EE5C8E420FD1641C64B280F8FC
:109320003740EB5C8B4202D1641C80F8374090F9E7
:1093300037300F2B1BDD0F2317E0434DEE5C434D01
:109340008E4202D0EE5C8E4211D1641E64B280F86F
:109350003740EB5C8B4202D1641E80F8374090F9B5
:1093600037406FF00E039C4201DA80F83730324B01
:1093700090F83F50393390F83740EC5490F83F3034
:109380005B1CDBB280F83F30062B01D380F83F2016
:1093900090F9394090F93B309C420ED190F93D4014
:1093A000A3420AD190F93A4090F93C309C4204D152
:1093B00090F93E40A34200D1012280F84F201F4A7D
:1093C00080F8401090F937501378214A012D0DDDB7
:1093D00014465E07A46804D544F0080403E028E0BE
:1093E00015E024F00804946080F83510B5F1FF3FD3
:1093F0000ADA5B07936802D523F0080301E043F023
:109400000803936080F83510F0BCFAF7A9B990F81A
:109410004F1001290DD1B0F8721043F60953491CC1
:1094200089B2A0F87210994203D9A0F8722080F88E
:109430004F20F0BC70470000140C002038010020C1
:10944000B8B80008BEB80008CAB80008D0B800080C
:10945000A402002010B502884188B0F908301144F8
:1094600009B281FB0313890B428041EA8341B0F9C1
:109470000420B0F9063082FB0332940444EA9332AC
:109480001144818010BD000030B52049204AB1F858
:109490006A301088C01A80B20F2836D31088A1F81D
:1094A0006A001C4D00204FF000432A5C940903D051
:1094B0000124B4EB921F24D1D20622D0164A52F8CE
:1094C00020201268134C123434F81040224201EB71
:1094D000000494F9722008D00A2A04DB0A6823FAEF
:1094E00000F4224308E0521C09E012F10A0F05DCE7
:1094F0000A6823FA00F4A2430A6002E0521E84F8CC
:109500007220401CC0B21128CFD330BDE805002026
:1095100048070020CCB30008CCB400082DE9F007C0
:109520007A497B480A8903889A1A92B2082A75D325
:1095300000880881A1F12C0042890AB1521E4281A3
:10954000744A92F82820802A68D302F03F020A70F9
:10955000C2890AB1521EC281B1F90620902A0CDBE1
:109560008A46FF2A09D08146C089002856D16A4818
:1095700000230078092805D005E0BDE8F00763481E
:1095800000F0C0B90823654A92F8EE500DB143F0DF
:1095900004036348817AC90701D043F00203D2F87B
:1095A00008C05FEA0C5101D543F0010317680021A0
:1095B0005C4EFC0302D596F8654004B18021C48856
:1095C0005FEA446801D541F040015FEA845801D563
:1095D00041F020015FEAC47801D041F01001007A27
:1095E000400701D541F008014F480078C00701D07D
:1095F00041F00401A00601D541F001010020012D38
:1096000000D1082096F870508DB992F84A20032AAC
:1096100005D0022A06D0012A07D008E072E040F007
:10962000030004E040F0020001E040F001007A078E
:1096300001D440F02000CCF3C0020025CCF3002C74
:10964000624502D13A0700D4042596F86F20012A1A
:1096500001D145F00105354A0027BC4612783E4647
:10966000C2F38102012A04D0022A04D0032A04D0C2
:1096700004E0022602E0042600E010262C4A6406DC
:109680000ED5224C1C342478240609D5147864069F
:1096900006D4284A40F6CC44926D6243140C05E08F
:1096A000B2F8B62040F699146243940B4FF00808C4
:1096B0008AF80A804FF061088AF80B808AF80C302B
:1096C0008AF80D108AF80E008AF80F508AF8107088
:1096D000270A4B4083F06901414069408AF81170C4
:1096E00079408AF81240614052468AF813C07140AE
:1096F0008AF8146051754FF4C871A9F80E10FF2054
:10970000AAF80600BDE8F00770470000F406002044
:1097100048070020E80500203F070020A4020020A1
:10972000000C0020580E0020B00A0020D0040020B9
:1097300038010020540900205D48816941F0FC0196
:1097400081614FF4A060FBF73DFFFAF72BFBF7F7C1
:1097500037FAFBF7AFFD002156A000F021F9584978
:109760000860FDF7EFF8FCF7E1FEFFF733FBFBF7CE
:109770000DFAFFF7BBFBFAF787FA524D4FF4005092
:10978000A5F81A01FCF7CEF8FCF782F800214FF497
:10979000FA5340F2EE220020401C80B29842FBD3E4
:1097A000491C89B29142F6D3474C002684F8726076
:1097B000F7F796F8F8F718FF42F21C202083401CB8
:1097C000608342F20320A08342F2AA00A080F8F74F
:1097D00011FCFEF737FC10223C493D48F6F7D3FC5C
:1097E00001F0F6F93B4C3D4FE08820F04000E0806E
:1097F0003948017821F020010170FA20F8814FF4F6
:109800009670A5F84200FFF749F835493548FBF74F
:10981000EAFF3548FCF70CF83448416A8847344879
:10982000416B8847FEF79EFD3248F9F7A3FAF8F737
:1098300013FC31494220C8803049C8603048F7F7EE
:109840006BFBA86820F48070A8603E71E088E0811E
:109850002089208260896082F9F70EFEF9F76AFD9F
:10986000FEF780FE01F034F9FFF7A8FB00F034FAB0
:10987000FFF70AFE00F0E4FFF9F750FBF8F716FCDB
:10988000FAF782FCFFF7FEF9FCF734FAFAF7A4F8CE
:10989000FAF7D6F800F0B2F8FFF740FE1548F9F7EE
:1098A00015F900F0A5FAFCF785FEF9F799FACDE76E
:1098B000001002406465765F63616E310000000055
:1098C0004C080020A402002038050020580E00207B
:1098D00028060020000C0020380100203C07002052
:1098E000000A0020D00900200C04002020000020E5
:1098F000CC0000203C0B002030070020400400205A
:10990000B00B0020F0B523490278B0F906400023DF
:109910001F4E31F81210FF2C18D0B0F904701E4DF4
:10992000BC4231DA00EBE40704F00704BF7AA74039
:109930008478FFB23CB190F801C0ACF1010C6445F1
:109940001FDA3C061DD455F822200DE056F82220DF
:10995000116012498A79521CD2B28A71022A02D34A
:109960008370C3808B71F0BD11608178491CC9B2CE
:10997000817042789142F6D38370C188491CC180BE
:10998000F0BD56F82220EFE755F822201160F4E7E9
:10999000ACB50008DEB3000854B50008C8060020C6
:1099A0002DE9F0410F4680460024124D124E08E08A
:1099B000286850F8240001684046F6F7F6FB38B1F5
:1099C000641CB4EBA60FF3DB6FF00100BDE8F0817F
:1099D000286850F824004068016829B13846884753
:1099E00028B16FF00200F1E76FF00500EEE72046C6
:1099F000ECE700007C08002004000000F0B561489E
:109A00006149B0F86C200B889A1A92B29C2A7BD3D9
:109A10000988A0F86C105D495D4F91F82A1001F09B
:109A2000070297F84A10022A00D1491E594C80F8C3
:109A30003E104FF00203E2884FF00001550401D5BB
:109A4000012236E0A489E50601D5062231E025078A
:109A500001D508222DE0550603D44F4D2D78AD06D3
:109A600001D5042225E0150501D5072221E01506C0
:109A700001D50A221DE0950601D50C2219E0150733
:109A800001D50B2215E0550701D4D50501D51022CB
:109A90000FE0D50601D505220BE0650703D4A50725
:109AA00001D4E40702D080F86E3007E0920403D5B9
:109AB000032280F86E2001E080F86E10374A384C9F
:109AC00092F820E0324A251FD2F808C02D4AB2F899
:109AD0007060721C92B2BEF1000F0DD02CF4000C1D
:109AE000C7F808C090F86E70B7B11E2F1AD090F862
:109AF0006F200AB325E007E04CF40006BE60A0F832
:109B000070200A2A01D22360F0BD142A01D22B60F2
:109B1000F0BDA0F87010F0BD2B60A0F8701080F8B8
:109B20006F10F0BD642E04D2A0F87020322AEED35C
:109B3000E9E7A0F87010EAE77F1C80F86F70A0F8E2
:109B4000701090F86F20012A10D0002AE9D0B0F8E8
:109B50007060761CB6B2A0F870601E2ED7D323605A
:109B60003C2EDED9521E80F86F20D2E7B0F870206C
:109B7000521C92B2A0F870202360C82AD1D980F874
:109B80006F10C6E7E805002048070020580E0020A7
:109B9000A4020020000C002038010020D004002086
:109BA000141C0140F0B54548B0F84810491C89B272
:109BB000A0F8481002297DD341490024A0F848406C
:109BC0000A78404B042A5BD04FF48041082A0BD01E
:109BD000A0F10C02B2F900208A4200DA1146B3F972
:109BE00084208A4200DA1146374A12698A4200DA32
:109BF00011B2418282881D8AC2EB8502334D12B2B6
:109C00002D78C5F381062D4D40F6D9467243B5F93E
:109C1000765092126A431213C26086681546C6EBEC
:109C2000C60642F3D102F60202EBA6328260C66C8F
:109C30001644C664B0F850707F1CBFB2A0F85070D4
:109C4000B7F5806F04D3B6120682A0F85040C46402
:109C5000C66A891AA6EB461740F2545207EB07175B
:109C60004A43A7EBC61602EB4602466A32444262FA
:109C7000B3F93430B2EB034F06DD1A04426206E05A
:109C80001349B1F90410AFE7002A00DA4462C16257
:109C9000104990F83D2091F838108A420DD080F894
:109CA0003D10B0F84210A0F84410B0F84010A0F8F1
:109CB000421000E001E0A0F84050F0BD380500205F
:109CC0003F070020A4020020F80D0020D00400204F
:109CD0000C0E00203801002015481649B0F85A2013
:109CE0000B889A1A92B20F2A20D30988A0F85A102A
:109CF000B0F900104FF48042C1EBC12141F3513162
:109D0000A0F86C100C490B78A0F10C01022B06D1C5
:109D1000B1F90030934202DA1B1D0B8000E00A808B
:109D20000021A0F8601020F85C1F428070470000FE
:109D300038050020480700203F0700204FF6FF723B
:109D400002EA800210F4404315480ED0B3F5804F6C
:109D500014D0B3F5004F4FEA122216D0C2F580732B
:109D600030F813305B424B8005E0120A30F81230B5
:109D70004B80C2F5807230F812000FE0120AC2F573
:109D8000807330F813304B8005E030F81230C2F5A4
:109D900080725B424B8030F812004042088070476E
:109DA000C8B10008104A518AD08A928A16384639BA
:109DB000A2F1110200D54942002A00DA52421144B0
:109DC000002800DA40420844084943F6284300B21C
:109DD000B1F936205A43921340F2D733584302EB7D
:109DE000A030C88670470000A4020020380500207B
:109DF000F0B5904990480A8903889A1A92B23E2A8F
:109E00001ED30088088101F138004FF4FA63428ABA
:109E10009A4202D2521C428200E04382874A92F860
:109E20002220802A0CD302F03F020A70B1F90620EA
:109E3000402A06DBFF2A04D0C2883AB1521EC280F3
:109E4000F0BDBDE8F0407B48FFF75CBD428A9A4216
:109E5000F6D307784FF0010E3A074FF0FF055BD5B8
:109E6000847A40F2DC52630708D444F0040383721E
:109E7000C28081F80BE081F80AE04CE04378072BC0
:109E800005D0032B03D0052B01D0062B07D1660686
:109E900005D444F040038372C280052239E0654A4C
:109EA0005FEA437C02F138024FF42076127A0DD536
:109EB0005FEAC26C0AD45FEA446C07D442F0100235
:109EC00002723A0628D4C680192222E0DF0709D0A0
:109ED000970707D4670605D442F002020272C680D3
:109EE000042216E09F0709D5170707D4670605D493
:109EF00042F008020272C68003220AE01B070BD55B
:109F0000530709D4630607D442F004020272C680E4
:109F10000B22CA728A72CD80494AB2F92230B2F954
:109F20001A7003F23D140022A74200DB0276414E74
:109F3000444C06F13806A479B6895FEAC46C06F190
:109F400001064FF4C874B6B213D58681B6F57A7F90
:109F500005D9017A21F0800101728281F0BD037A76
:109F60001E06FBD4828143F080020272C48011205D
:109F700035E09F4216DA037E052B13D28681B6F5B3
:109F8000487F04D98281027A22F040020272027A6A
:109F90005606E3D45B1C037642F040020272C48092
:109FA00002201CE0284B1C89C4F3C006C4F3002720
:109FB00040F2EE24BE4216D11E78360713D4427EFC
:109FC000012ACBD1428BB2F5167F02D2521C4283BA
:109FD000F0BD827A42F002028272C4800F20C87201
:109FE0008872CD80F0BD93F811714FF40046012FB7
:109FF00018D1164F41F6583C7F6C674512DD83F847
:10A0000010E1134B1E60C38AA34202D25B1CC382C1
:10A01000F0BD4FF4FA73C3801C23CB728B72CD80DA
:10A02000C282F0BDC2820A4883F81021001F066078
:10A03000F0BD0000D806002048070020E8050020F9
:10A04000D0040020000C0020A402002038010020D1
:10A05000140801402DE9F05FDFF8FCB3FF489BF8DE
:10A060001830011D0A1DFE4C012B5FD0B4F85E3084
:10A070000380B4F860000880B4F862001080FDF737
:10A080002FFBDFF8E083F84D49F2CD32B8F91E001E
:10A09000A883B8F9201043F6CC4C00EB41015143A2
:10A0A0000914E983B5F92230B5F9206001FB03F208
:10A0B00000FB062242F38F326A82B5F918707143B1
:10A0C00007FB0CF740F2333CBF1302FB0CF207EB2B
:10A0D000A23200FB13102A8340F38F30A882B5F917
:10A0E0001A1043F6AE72514300EB0012891302EBD3
:10A0F0008010DE4F01EBA030DD4E6883786C30605D
:10A10000316930468847DB49308948800846FDF789
:10A11000C9FBD94E4FF000094FF0010A30780828EA
:10A120000DD0698F2982042833D01BE0B4F8643045
:10A130000380B4F866000880B4F868009EE7CF4852
:10A1400090F93710491C022921D890F8741019B1E0
:10A15000B5F85A00288205E0698F2982A5F85A10BF
:10A1600080F874A0B5F91410B5F90A00C44AF8F7DC
:10A1700051FBE862B4F91A11884204DDC048E96273
:10A18000027C914081623078042816D00CE0688F00
:10A19000E0E7D8F824000014E862E07B04280CD043
:10A1A000C5F82C9086F80090B54AB5F91210B5F9AB
:10A1B0000800303AF8F72EFB02E0B87AF0B3B14865
:10A1C000A862A94DAE4E443EA86A3060E86A70604D
:10A1D00030461035FBF76AFD2888A5F14C01FFF7E2
:10A1E000ADFDA5F15C08D8F81010C8F86C10B5F9F1
:10A1F0001020B068B5F9121000FB02F7F36848436D
:10A2000003FB117646F38F3703FB0200AF8740F361
:10A210008F36EE879C4D28466F80AE80FDF784FF19
:10A22000287F08F11405012833D0704242104DF602
:10A23000B35047436A803914298000E026E0404645
:10A24000A8F8006053184380511AA8F8041084F845
:10A250000C90B8F90030002B01DD84F80CA0B8F99F
:10A260000200002802DD217B891C2173B8F904203B
:10A27000002A02DD217B091D2173217B072920D2C1
:10A28000DFE801F01F1B3418301D32004FF4AF70AF
:10A2900096E77D48B0F9203059424A106A80B0F9FB
:10A2A0001E004DF6B3514843011429804046A8F8DA
:10A2B0000030C7E784F80DA003E0022100E003218D
:10A2C0006173DFF8A4A1714E714F9AF80010012953
:10A2D000617B0DD0072972D2DFE801F071FCFBFA37
:10A2E000F9F8F7000421EBE70521E9E70621E7E7A4
:10A2F0000729F0D2DFE801F063042F6489D5EF006D
:10A3000001461846FBF756FA2860B5F9020040F6F8
:10A310008151484381136980B5F9000040F68152AC
:10A320005043801328800A18A2F68152B8F80A30E8
:10A330005242C3EB620212B2A8F80820002A01DCE4
:10A34000A8F80890B8F80820A4F862201144A4F8EE
:10A35000601008446DE1404201B2504200B2FBF788
:10A3600029FA2860B5F9020040F68151484381136B
:10A370006980B5F9000040F681525043801328806F
:10A380000A18A2F68152B8F80A305242C3EB6202B0
:10A3900012B2A8F80820002A01DCA8F80890B8F842
:10A3A0000820A4F862201144A4F85E1008446EE16D
:10A3B0003046F6F763FC01231A460721CAE0D4E0D1
:10A3C00019461046FBF7F6F92860B5F9020040F689
:10A3D0008151484380136880B5F9001040F68152DE
:10A3E0005143891329804218A2F68152B8F80A30E5
:10A3F0005242C3EB620212B2A8F80820002A01DC24
:10A40000A8F80890B8F8082068E15942404209B21B
:10A4100000B2FBF7CFF92860B5F9020040F6815190
:10A42000484380136880B5F9001040F681525143CB
:10A43000891329804218A2F68152B8F80A30524294
:10A44000C3EB620212B2A8F80820002A01DCA8F8C7
:10A450000890B8F8082071E13C0B0020342C014032
:10A46000A4020020380500204C0000203801002004
:10A4700040040020FC0300203F070020140C0020B3
:10A48000000A0020A2FEFFFF700B00200024014004
:10A49000002801403046F6F7F1FB01231A4605215A
:10A4A00058E01146FBF786F92860B5F9020040F63E
:10A4B0008151484380136880B5F9001040F68152FD
:10A4C000514389132980421806E076E14AE11BE1F5
:10A4D000ECE0BCE08FE010E0A2F68152B8F80A3060
:10A4E0005242C3EB620212B2A8F80820002A01DC33
:10A4F000A8F80890B8F808204BE1504201B2584241
:10A5000000B2FBF757F92860B5F9020040F6815117
:10A51000484380136880B5F9001040F681525143DA
:10A52000891329804218A2F68152B8F80A305242A3
:10A53000C3EB620212B2A8F80820002A01DCA8F8D6
:10A540000890B8F8082052E13046F6F797FB01234F
:10A550001A4606213846F6F791FB01213046F6F7F8
:10A5600003FB01213846F6F7FFFABAF80800ABF80A
:10A570000000BAF80A00ABF80200BAF81000ABF815
:10A58000040055465E46AB48F8F702FBB4F85E009F
:10A59000F1880844A4F86400B4F8600031890844E4
:10A5A000A4F86600B4F8620071890844A4F8680051
:10A5B000317EA148012978D034F85E1F018061887E
:10A5C0004180A18881809C49028808310A804288A4
:10A5D0004A80808888809848896A0830884795F83A
:10A5E0003E0000287ED0F7F729FF15F83E0F401EE9
:10A5F0002870BDE8F09F01461846FBF7DBF828609D
:10A60000B5F9020040F68151484380136880B5F9DE
:10A61000001040F68152514389134218A2F681522C
:10A62000524252082980A4F862201044A4F8600025
:10A630000844A4F85E0000213046F6F795FA0021A0
:10A640003846F6F791FA01231A460621B0E6404251
:10A6500001B2504200B2FBF7ADF82860B5F9020034
:10A6600040F68151484380136880B5F9001040F6E8
:10A670008152514389134218A2F681525242520824
:10A680002980A4F862201044A4F85E000844A4F8CD
:10A69000600000213046F6F767FA00213846F6F7E9
:10A6A00063FA01231A46052182E6B4E019461046F2
:10A6B000FBF780F82860B5F9020040F68151484365
:10A6C00080136880B5F9001040F681525143891318
:10A6D0004218A2F68152524229805208A4F85E2004
:10A6E000104400E09AE0A4F862000844A4F8600076
:10A6F00000213046F6F738FA00213846F6F734FAEA
:10A7000001231A460721C5E65942404209B200B268
:10A71000FBF750F82860B5F9020040F68151484334
:10A7200080136880B5F9001040F6815251438913B7
:10A730004218A2F68152524229805208A4F85E20A3
:10A740001044A4F860000844A4F8620000213046D8
:10A75000F6F70AFA00213846F6F706FA01231A46F8
:10A76000062197E61146FBF725F82860B5F90200A7
:10A7700040F68151484380136880B5F9001040F6D7
:10A780008152514389134218A2F6815252422980C4
:10A790005208A4F860201044A4F85E000844A4F80D
:10A7A000620000213046F6F7DFF900213846F6F75F
:10A7B000DBF901231A460521C6E6504201B2584290
:10A7C00000B2FAF7F7FF2860B5F9020040F68151B0
:10A7D000484380136880B5F9001040F68152514318
:10A7E00089134218A2F68152524229805208A4F8D5
:10A7F00060201044A4F862000844A4F85E00002120
:10A800003046F6F7B1F900213846F6F7ADF90123E5
:10A810001A46072198E634F8641FCFE607480088F7
:10A82000A0F5D04168393FF4E4AEBDE8F05FF8F739
:10A830005DBC00003C0B002018000020182C0140DB
:10A840002DE9F041944C9548B4F862100288511AF1
:10A8500089B20F296FD30088A4F86200904800885D
:10A86000DFF84082C0074FF000054FF0010741D0EC
:10A870008B4AD4E90C1024321388B1EB530F02D267
:10A880001288511A08444FF4F371884200D20846E6
:10A890008549B1FBF0F0616CC1F3510108440646F3
:10A8A0006064F5F7C8FD0022804BF5F730FD4FF0EE
:10A8B00040427F4BF5F72BFD0E22F5F797FDF5F79C
:10A8C000F1FDA4F8AC0094F86D00401CC0B284F80F
:10A8D0006D00082834D3704898F84A20001F037888
:10A8E0009A4201D002704580724A1378724A23B1AD
:10A8F000458021E06564256569E0D8F89810A1F5E8
:10A90000FA618E4211DDE16D8B1C9E4205DDB0F9CE
:10A9100002100A290DDA491C06E08E4205DAB0F968
:10A920000210002908DD491E4180B0F902000A2802
:10A9300002DB177001E0ABE01570E66584F86D503E
:10A940005E484FF4A5420178C1F38101012962D02C
:10A9500044F25063A4F80830A4F8A820B0F92430D9
:10A9600021894B439B13A4F8A430B0F90E00D4F80E
:10A9700050C07043B0FBF1F35149CCEBCC0C4FEA23
:10A98000CC2C0988C3F3D10303EB9C33B0032365BC
:10A99000B0FBF1F14B4BC908B3F846C0CCEBCC0C83
:10A9A0004FEACC2C01EB9C31A3F84610F117890338
:10A9B00041EA96410023F5F7B5FBB4F8AA10C1EBC4
:10A9C000C101C902C00800EB9130A4F8AA00616C73
:10A9D000206F0844206794F87420521CD2B284F887
:10A9E0007420082A05D3C008A4F8760084F87450AF
:10A9F00025673548C3885A0605D498F80F20022ADF
:10AA00000DD0A4F88A50244894F83F20B8300C2A7E
:10AA100028D2C57427E045F6C05121819CE794F8FF
:10AA2000382094F88E60B2420CD084F88E2094F8CE
:10AA30003D2002F00106C2F34002964202D1A4F882
:10AA40008A5005E0B4F88A2040F6B836B24205D202
:10AA5000B4F88A00401CA4F88A00D4E743F08002CE
:10AA6000C280D0E7C774194B0E4C41F2482693F8C8
:10AA70003C30B4F8864041F2504C0C2A0AD3B14223
:10AA800008DB012B06D0614502DD002C00D1877464
:10AA9000BDE8F0818574FBE73801002048070020FD
:10AAA00000040040A40200204564BD0100209C4039
:10AAB000133B3340FA030020FB030020D0040020A6
:10AAC00030010020300A0020000C00203805002052
:10AAD00070B5394C394821880288511A89B23E290B
:10AAE0004DD30088364E20803649307806F1140563
:10AAF00018B3488B80002880E96828468847B5F954
:10AB000004003149FCF79FFD304A60804FF48045D6
:10AB1000D3884FF000015E0737D4B0F5DC5F2FDD3E
:10AB2000E079401CC0B2E0710A283ED343F40040F3
:10AB300040F00400D080A16036E0888B204A80007D
:10AB4000121D1080888B80005080888B800000B29E
:10AB500090804A8B92002A804A8B92006A80498BAF
:10AB60008900A98018497C31FCF76DFDA080B5F9FA
:10AB700004001549FCF767FD60800120307070BD4E
:10AB800023F40040A560D0800EE043F4004343F07E
:10AB90000403A160D380B0F5B45F06DC23F4004069
:10ABA00020F00400D080A560E171D4E90201884260
:10ABB00000DB0846206170BDF80D0020480700202A
:10ABC00094060020A4020020C0B70008000C00205A
:10ABD00005494FF48040C860886008610348C18817
:10ABE00021F48271C1807047F80D0020000C002014
:10ABF0002DE9F041384C394E394F207841F233314C
:10AC0000C2074FF000050CD0A28962B394F9070087
:10AC1000002800DA4042C0B2032829D240F2AE70C8
:10AC20002AE0A570E5732F4AE571A58192F83830C6
:10AC3000237220F00800A18040F002002070BD8641
:10AC40007560B560F560116D490005D041F684610D
:10AC5000A18140F010002070C0B240F001002070CF
:10AC60006574BDE8F081658120F01000207015E06A
:10AC7000042803D240F6510060810FE0052802D27B
:10AC800040F69910F8E740F6CC42062803D307288F
:10AC900001D3082801D2628100E0618197F8A10008
:10ACA00098B9B088102301B2B4F90A003622FBF734
:10ACB00037FD7060F168401AB1680844B060B6F9B9
:10ACC00000104843C013F060B886B88E10B1012060
:10ACD000A070C6E7A570C4E70C0E0020B8060020DF
:10ACE000A4020020380100202DE9F041554C2678BF
:10ACF000F0077CD05448217A544D90F838008142B6
:10AD00007BD0534A2346DFF84CC1575C93F90E20A1
:10AD100093F90730874203D01CF80170874213D1A2
:10AD200046F002065B1C26705BB2E3711CF8011052
:10AD3000814201D15B1CE37194F90710062901DD02
:10AD40000621E171521C1CE0434F17F801C0434F2C
:10AD5000844503D017F801C0844513D126F00206BC
:10AD60005B1E26705BB2E371795C814201D15B1E90
:10AD7000E37194F907306FF005018B4200DAE1715D
:10AD8000521EA273207294F907108A1C042A02D959
:10AD900041F68462A2812C4A012912780ADD2B4BEC
:10ADA00056079B6802D543F0080301E023F008032F
:10ADB000AB606070B1F1FF3F09DA5107A96802D5B5
:10ADC00021F0080101E041F00801A9606070F8F786
:10ADD000C7FCA078012810D121488068A3280CDA8C
:10ADE00094F90700022803DD0220E07105E01EE06F
:10ADF0006FF00101884200DAE171A089002630B1CC
:10AE0000401E0004000CA08101D1E671A673E87B0E
:10AE100004280CD0B5F93410512341220020FBF74F
:10AE20007FFCA886002802D1E07B10B1A670BDE8A7
:10AE3000F0810C4806700C480670207820F0010064
:10AE40002070F4E70C0E002038010020A40200203E
:10AE5000B8B80008BEB80008CAB80008D0B80008E2
:10AE6000380500205C0700203F070020F0B415469D
:10AE70000D4A0E464FF0FF31B0EBA20F12DA002858
:10AE800010DB0A49096851F82000406844682CB179
:10AE900029463046A446F0BC1A4660476FF00500CC
:10AEA000F0BC70470846FBE7040000007C08002067
:10AEB000173E573CBB3A3E39DD3794366135413455
:10AEC00033333532443161308A2FBD2EFB2D412D75
:10AED000CC1C58585868991958585868331300565C
:10AEE00095130054B61300525A140050FD14004E2E
:10AEF000A115004C4516004A761600486C1700460E
:10AF000072180044BA190042741B0040911D003EA3
:10AF1000B420003C9F22003AE1220038532300363F
:10AF20008B240034812500322B2700302028002E6E
:10AF30005829002CB02A002A9B2C0028D22D00264C
:10AF40007C2F00242631002202330020FD34001E15
:10AF50005C37001CCC3C001A873E0018BE3F001630
:10AF60000040001400400012004000100040000E9D
:10AF70000040000C0040000A0040000800400006AD
:10AF800000400004004000020040000001020304F1
:10AF9000050005000102030401040003050200008E
:10AFA000F001000036010000F8000000BA000000C7
:10AFB0007C0000007C0000007C000000C91C9C1983
:10AFC000991CCC199C1CC9190000290052007B0057
:10AFD000A400CC00F5001E01470170019901C201D7
:10AFE000EA0113023C0265028E02B602DF02080388
:10AFF000300359038203AA03D303FB0324044C0444
:10B0000075049D04C504EE0416053E0567058F050D
:10B01000B705DF0507062F0657067F06A706CE06EB
:10B02000F6061E0746076D079507BC07E4070B08E1
:10B03000320859088108A808CF08F6081D094409F4
:10B040006A099109B809DE09050A2B0A520A780A29
:10B050009E0AC40AEA0A100B360B5C0B820BA80B83
:10B06000CD0BF30B180C3E0C630C880CAD0CD20C02
:10B07000F70C1C0D410D650D8A0DAF0DD30DF70DAD
:10B080001C0E400E640E880EAC0ECF0EF30E170F82
:10B090003A0F5E0F810FA40FC70FEA0F0D1030108B
:10B0A000531075109810BA10DD10FF1021114311C4
:10B0B00065118711A911CA11EC110D122E1250122F
:10B0C00071129212B312D412F412151336135613CE
:10B0D00076139613B713D713F613161436145614A3
:10B0E00075149414B414D314F214111530154E15AC
:10B0F0006D158C15AA15C815E715051623164116EA
:10B100005F167C169A16B716D516F2160F172C175F
:10B11000491766178317A017BC17D917F517111809
:10B120002E184A18661881189D18B918D418F018E6
:10B130000B19261942195D1978199219AD19C819F8
:10B14000E219FD19171A311A4C1A661A801A991A3F
:10B15000B31ACD1AE61A001B191B331B4C1B651BB7
:10B160007E1B971BAF1BC81BE11BF91B121C2A1C63
:10B17000421C5A1C721C8A1CA21CBA1CD21CE91C40
:10B18000011D181D301D471D5E1D751D8C1DA31D45
:10B19000BA1DD01DE71DFD1D141E2A1E401E571E80
:10B1A0006D1E831E981EAE1EC41EDA1EEF1E051FE6
:10B1B0001A1F2F1F451F5A1F6F1F841F991FAE1F75
:10B1C000C21FD71FEC1F002000006400C9002D0122
:10B1D0009201F7015B02C00224038903ED035204CC
:10B1E000B6041A057F05E3054706AB060F0773078C
:10B1F000D7073B089F0802096609C9092D0A900A6A
:10B20000F30A560BB90B1C0C7F0CE20C440DA60D77
:10B21000090E6B0ECD0E2F0F900FF20F5310B410BE
:10B2200015117611D71138129812F8125813B81355
:10B2300018147714D61435159415F3155116B01645
:10B240000E176B17C91726188318E0183D1999199E
:10B25000F519511AAD1A081B631BBE1B181C731C71
:10B26000CD1C261D801DD91D321E8A1EE31E3B1FCC
:10B27000921FEA1F41209820EE2044219A21EF21BD
:10B2800045229922EE2242239623E9233C248F244F
:10B29000E22434258525D72528267826C826182790
:10B2A0006827B72706285428A228EF283D2989298E
:10B2B000D629222A6D2AB82A032B4D2B972BE12B56
:10B2C0002A2C722CBB2C022D4A2D912DD72D1D2EF0
:10B2D000632EA82EEC2E302F742FB82FFA2F3D306E
:10B2E0007F30C030013141318131C13100323F32D4
:10B2F0007D32BA32F73234337033AC33E733223431
:10B300005C349534CE3407353F357735AE35E4358A
:10B310001A3650368536B936ED36203753378637EC
:10B32000B737E937193849387938A838D73805395F
:10B3300032395F398B39B739E2390D3A373A603AE9
:10B34000893AB23ADA3A013B283B4E3B733B983B91
:10B35000BD3BE03B043C263C483C6A3C8B3CAB3C60
:10B36000CB3CEA3C093D273D443D613D7D3D993D57
:10B37000B43DCE3DE83D013E1A3E323E493E603E80
:10B38000763E8C3EA13EB53EC93EDC3EEF3E013FDF
:10B39000123F233F333F433F513F603F6E3F7B3F70
:10B3A000873F933F9E3FA93FB33FBC3FC53FCD3F43
:10B3B000D53FDC3FE23FE83FED3FF13FF53FF93F4E
:10B3C000FB3FFD3FFF3FFF3FFF3F0000E0203420F9
:10B3D000002020E02020202337202620210000808C
:10B3E000020004000800100000020004000804002D
:10B3F000000200040008001000200040008004004B
:10B40000000000800000004000000020000000104C
:10B41000000000080000000400000002000000011D
:10B42000000080000000400000002000000010002C
:10B4300000000800000004000000020000000100FD
:10B440000080000000080140000C0140000C014099
:10B45000000C0140000C0140000C0140000C0140B8
:10B46000000C01400010014000100140001001409C
:10B470000010014000100140001001400010014088
:10B48000001001400014014004080140040C014078
:10B49000040C0140040C0140040C0140040C014068
:10B4A000040C0140040C0140041001400410014050
:10B4B0000410014004100140041001400410014038
:10B4C0000410014004100140041401400808014028
:10B4D000080C0140080C0140080C0140080C014018
:10B4E000080C0140080C0140080C01400810014004
:10B4F00008100140081001400810014008100140E8
:10B5000008100140081001400810014008140140D3
:10B510000C0801400C0C01400C0C01400C0C0140CB
:10B520000C0C01400C0C01400C0C01400C0C0140B7
:10B530000C1001400C1001400C1001400C10014097
:10B540000C1001400C1001400C1001400C10014087
:10B550000C14014010080140100C0140100C014077
:10B56000100C0140100C0140100C0140100C014067
:10B57000100C01401010014010100140101001404B
:10B580001010014010100140101001401010014037
:10B5900010100140101401400000000000000000E5
:10B5A000000000000000000000000000140801403E
:10B5B000140C0140140C0140140C0140140C014007
:10B5C000140C0140140C0140140C014014100140F3
:10B5D00014100140141001401410014014100140D7
:10B5E00014100140141001401410014014140140C3
:10B5F000000000000000000000000000000000004B
:10B6000000000000FFFFFF0F0FFFFFFFFFF0FFFF35
:10B61000FF0FFFFFFFFFF0FF0FFFFFFFFFF0FFFF38
:10B62000FF0FFFFFFFF0FFFF0FFFFFFFFFF0FFFF28
:10B63000FF0FFFFFFFFFF0FFFFFF0FFFFFFFFFF018
:10B64000FFFFFF0FFFF0FFFF000000404000000081
:10B650000004000000400000000004004000000062
:10B660000004000000400000000400004000000052
:10B670000004000000400000000004000000400042
:10B6800000000004000000400004000000000080F2
:10B69000800000000008000000800000000008009A
:10B6A000800000000008000000800000000800008A
:10B6B000800000000008000000800000000008007A
:10B6C000000080000000000800000080000800006A
:10B6D0000000002020000000000200000020000008
:10B6E0000000020020000000000200000020000016
:10B6F0000002000020000000000200000020000006
:10B7000000000200000020000000000200000020F5
:10B710000002000000000060600000000006000061
:10B72000006000000000060060000000000600004D
:10B73000006000000006000060000000000600003D
:10B74000006000000000060000006000000000062D
:10B7500000000060000600000080020004000800F5
:10B7600010000002000400080400000200040008A9
:10B77000001000200040008004000000FF7FFFFF59
:10B78000FDFFFFFFFBFFFFFFF7FFFFFFEFFFFFFFE7
:10B79000FFFDFFFFFFFBFFFFFFF7FFFFFBFFFFFFCB
:10B7A000FFFDFFFFFFFBFFFFFFF7FFFFFFEFFFFFC7
:10B7B000FFDFFFFFFFBFFFFFFF7FFFFFFBFFFFFF7D
:10B7C000401FFC02001E5A03C01CC403801B3C0423
:10B7D000401AC60400196305C01717068016E40650
:10B7E0004015CD070014D708C012050A80115B0B65
:10B7F0004010DD0C000F900EC00D7510800C9012E3
:10B80000400BE014000A6517C0081C1A8007FD1CD5
:10B810004006002000051823C003372680024E2969
:10B8200040014C2C0000242FC0FEC73180FD2E3477
:10B8300000FB2D3880F81C3B00F6003C8025151AD3
:10B8400040249A1B00231E1DC021B81E80205D20AD
:10B85000401F0C22001EC223C01C7E25801B3327E4
:10B86000401AFB280019B72AC0176D2C8016192E14
:10B870004015B92F00144731C012C9328011353438
:10B8800040108B35000FCA36C00DF037800CFE38E3
:10B89000400BF439000AD23AC008983B8007473C75
:10B8A0004006E13C0005673DC003DA3D80023E3EB4
:10B8B0004001923E0000143F010203040500020310
:10B8C0000405000103040500010205000102030450
:10B8D00004050001020355050010AA1A5525003081
:10B8E000AA3A0000AA0A55150020AA2A5535FF3F9A
:10B8F0006465765F63616E3100000000FD890008B9
:10B90000AD8B0008298B000859890008218900089F
:10B9100000000000F0B80008FCB8000840B90008BA
:10B92000000000208C080000000700086CBA000826
:10B930008C0800203C1500005485000814B900084C
:10B9400001441335401B084904211355152A4006AC
:10B95000190801A713AF5A1B08D5041ACF040124F4
:10B9600023286E420117020604050103148020FFFC
:10B970008BAA0A0201A415AA0A551500085920AA83
:10B980002A5535FF3F073103010504060203127CE7
:10B990001573FFFF04FF808001012D025F64021315
:10B9A0000A13558C52081201100C050406020301FB
:10B9B0000103070505280B01020304020607030320
:10B9C000040C3D0706040509191F19190431050661
:10B9D000060B14AA1A02312E40FD39692602110401
:10B9E0002F405F020C26405B262ACD5515551512B7
:10B9F0003902017F0316D0071AFF01013B0261AA39
:10BA00000C10080108A834993F33135594391CA928
:10BA1000100916E891220312100A17401C12600A3E
:10BA200016901B011AA2646B698C94012199D001B4
:10BA30009A5A14021AC802CBD007023A19164902C0
:10BA4000892612C8DA01DA1AFF01C1227D130D021C
:10BA500012103AFA0812081CF401010812062BE829
:0CBA6000031012021B3CB915B1000000DD
:020000040800F2
:10FC00004A46545A594D46312D4E3330202020203B
:10FC1000050406020301AA0AAA0AAA0AAA0AAA0A4B
:10FC2000AA0ADE3F00100000FF0131000301664612
:10FC300000400040513800400040004000400101B9
:10FC4000004000407A3B082708270827FF0033338D
:10FC50000201401F00016626B81E6626FFFFFFFF57
:10FC6000FFFF01010100010000000300000202008B
:04FC70000000AA5591
:04000005080000ED02
:00000001FF
